:020000040800F2
:10500000101C0020D5500008E988000845800008E1
:105010000000000000000000000000000000000090
:1050200000000000000000000000000035970008AC
:105030000000000000000000B19000087198000816
:10504000E7500008E7500008E7500008E750000864
:10505000E7500008155D0008E7500008E750000819
:1050600000000000E75000083D5C0008E750000821
:10507000E75000085985000800000000E7500008CC
:1050800000000000E75000080000000000000000E1
:10509000E750000800000000E7500008E750000853
:1050A000E7500008E7500008E750000859A1000841
:1050B000E7500008E7500008000000000000000072
:1050C0000348854600F0E8FC00480047CDB40008DE
:1050D000101C00200448804704480047FEE7FEE714
:1050E000FEE7FEE7FEE7FEE70D990008C150000865
:1050F00030B50B46014600202022012409E00D4670
:10510000D5409D4205D31D469540491B25469540F7
:1051100040191546521E002DF1DC30BDF0B51FB40C
:105120000646002082B005464024019100901BE015
:10513000019922460F46304600F098FB049A059BE1
:10514000801A994110D310461946224600F07EFB82
:10515000361A8F410197224601200021009F00F05E
:1051600075FB38184D4100902046641E0028DFDC96
:10517000019B00982946324607B0F0BD03460B4319
:105180009B0703D009E008C9121F08C0042AFAD2FD
:1051900003E00B780370401C491C521EF9D2704783
:1051A000D2B201E00270401C491EFBD270470022BF
:1051B000F6E710B513460A4604461946FFF7F0FF16
:1051C000204610BD30B504460020034600E05B1CBD
:1051D000934203D2E05CCD5C401BF8D030BDF8B503
:1051E00002464A40D40F42004B0052085B089A42E4
:1051F00002D20246084611464A0023D0C30D4A0097
:10520000DDB2120EAD1A202D35DA49020126490A07
:10521000F6058A19002C00D0524220214F1B11465E
:10522000B9402A411018C20D9A4221D0002C17D043
:10523000012D08DCDA05801AD20F8019D207DBB203
:1052400000F040FBF8BDDA05801A012340001B0680
:10525000C01880185A428018CA0F1043490007E04E
:105260004908C2071143DA05801A801940088018DE
:1052700000F020FBF8BD61000122511A001BF7E786
:105280000122D2075140AAE70122D2075040A6E7E7
:1052900070B502464A40D50F40004A00ED0740086D
:1052A0005208002814D0002A12D0C40DD30D410298
:1052B0000120C0055202490A520AE41A09181218BC
:1052C0007D34914201D3641C00E04900002C01DAD6
:1052D000002070BD0023914201D3891A0343400886
:1052E00049000028F7D100290AD0914202D10121BA
:1052F000C90705E0914201D2012101E00121C94322
:10530000E005C018401900F0D5FA70BD420005D084
:105310004200120E52428A4201DB00207047C9054A
:1053200008187047F0B507460846584087B0C00FC8
:10533000049048000E46590040084908BC1A8841AC
:1053400005D2384631461E4617460B4602465800DF
:10535000400810434CD0300D039040055900400DDB
:10536000490D0590401A0290402872DA1803012175
:10537000000B09050843019004980092002805D00D
:1053800001995242002088410092019002984021E8
:105390000A1A0199009800F059FA05460C466B4626
:1053A00007CB00F074FAC0197141039A0E0D002367
:1053B000D71756401A467A40164344D0049A002A1A
:1053C0002DD0029A012A039A15DC1205C01A9141C8
:1053D00001263605001C7141D20F059ED2070093AD
:1053E000019202962A46234600F0B2FA07B0F0BDB9
:1053F00038463146FAE71605224A0F46B218C01A57
:10540000B74101210905001C4F4100187F41114699
:1054100018187941E20F10436D19644113E0E20757
:105420006D0815436408C2071443039A0126120548
:10543000C01A91413605001C7141CE074008304327
:105440004908C01851412A46234600F074FACDE7B6
:10545000FFE7049801224000C117121A00238B4174
:1054600004983146C417381AA141EEE730B401243C
:10547000E407634030BC55E730B40124E4076140E1
:1054800030BC4FE70000E0FFF0B51FB488B00B99C7
:105490000998002448400999C00F4900490809911A
:1054A000C0070B990090490049080B910999089889
:1054B000A64608431CD00B990A98084318D00998AF
:1054C00001244000420D4800410D099824050003C5
:1054D000000B204309900B980003000B20430B9016
:1054E00050181C494018002201901446104605E04F
:1054F000002001460DB0F0BD032801DA034600E0AC
:1055000003239C46C11A0AAE0AE05F0008ADED5BBA
:105510004F00F75B7D430027AA187C41491C5B1EA6
:105520006145F2DD410004AB5A522104120C0A43DA
:10553000240C401C0828DFDB01980290009970467B
:1055400001910090059B049A0799069800F000FAD3
:10555000D0E700000DFCFFFFF0B50C465C4085B0C5
:10556000E40FE40703944C000026640859009446B5
:10557000490802460296224321D062460A431ED0C1
:105580006200570D4A000E032303550D0124024605
:105590002C492405781B1B0B360B4018234326434C
:1055A000614600901C46501AB44103D30098401C39
:1055B000009002E0921800985B41002803DA002076
:1055C000014605B0F0BD00200121090507468646C9
:1055D00011E064461D46141BB54106D36546521BB7
:1055E000B341744607430C43A646CD07400849081B
:1055F000284392185B4105460D43EAD110461843F3
:1056000013D06046194650407140084306D06046AA
:10561000101AB34106D20122002306E00022012322
:10562000DB0702E00122D2435310009874460105C3
:10563000381C6141029C039D0019694100F07BF90F
:10564000BFE70000FD03000070B54B005B0803439B
:105650000BD04B005C0D002633466542B341D41796
:10566000AD1AA34102DB0020014670BD12053018BF
:10567000514170BDC217C10F504010B54018CA0744
:105680009623002100F01EF910BD10B500229623CC
:10569000114600F017F910BD0EB5C217C10F5040EA
:1056A000CA0740180021054B0293019200910A4657
:1056B0000B4600F04DF903B000BD000033040000BC
:1056C0000EB505490291002100910A460B46019151
:1056D00000F03EF903B000BD330400004100400279
:1056E0000122400AD205090E80187F2901DA002024
:1056F0007047962903DC9622511AC84070479639A4
:105700008840704770B5CD0F4A0009030123090B8B
:105710001B0519430B4BED070024520D9A4201DA89
:10572000002070BD074B34339A4203DC9A1A00F014
:105730009DF802E00449511888402C43F1D04042C2
:1057400070BD0000FF030000CDFBFFFF4A0009030E
:105750000123090B1B051943094B10B5520D9A4241
:1057600001DA002010BD064B34339A4203DC9A1A4A
:1057700000F07CF810BD03495118884010BD0000AE
:10578000FF030000CDFBFFFFC20FD207400040081F
:105790000BD0C10D0723DB01C91840020905400ADF
:1057A0001143C2084007114370470020014670476B
:1057B00010B5002904DB0124E40740428C41214656
:1057C000002B04DB1C460123DB075242A3418B4222
:1057D00000D1824210BD000010B5002904DB012475
:1057E000E40740428C412146002B04DB1C46012388
:1057F000DB075242A341994200D1904210BD000004
:10580000CB0FDB07490010B5490802460A4307D011
:105810000A0D07240903E401090B121B002A01DC0D
:10582000002010BDC900440F0C43C100E018D20590
:10583000801800F03FF810BD0122D207002800DBDD
:10584000101A002900DB511A8142704710B5202A36
:1058500004DB0146203A9140002010BD91402023F6
:105860009C1A0346E3401943904010BD10B5202A0E
:1058700004DB0846203AD040002110BD0B46D3403F
:10588000D0402024A21A91400843194610BD10B5FB
:10589000202A06DBCB170846203A1041C1170B43DC
:1058A00006E00B461341D0402024A21A9140084341
:1058B000194610BD002904DA401C490001D14008F6
:1058C0004000704770B40024050C05D1102400047A
:1058D00002D1002921D01124050E01D10002083483
:1058E000050F01D10001241D850F01D18000A41CEA
:1058F000002801DB4000641C002908D020252E1B55
:105900000D46F540A14000D001212943084301067E
:105910001B1B000ADB1D02D5002070BC7047DB0595
:10592000181880180029F8DA401C4900F5D170BC1D
:1059300040084000704710B5002B08DA0024401CD6
:10594000614192185B411A4301D14008400010BDEB
:10595000F0B51FB482B005460C0003D0084604F031
:10596000AFFC02E004F0ACFC20300246009021467F
:105970002846FFF76BFF049B059A04460F46184321
:105980001143084314D0184610431BD000984021FF
:105990000A1A18460599FFF769FF05460E46009A50
:1059A00005990498FFF752FF084305D0012004E051
:1059B0002046394607B0F0BD0020C11705430E430D
:1059C0002C43374300990E986305401A7905E40A81
:1059D00000220C43FD0A0A3002D500200146E9E707
:1059E0000105101969410C9C0D9D00196941FFF7D3
:1059F000A2FFDFE7FEB500231A461B1A8A4103DB2C
:105A00000020014603B0F0BD4A000D0301212D0B1B
:105A10000905520D0D43D10702D100186D41521EE8
:105A20005110FF31FF310131002704463E46384610
:105A3000009701910246012100200905FFF716FF9A
:105A4000C3197141F818324684468E464A41614670
:105A50002846611A904104D36046241A954176463F
:105A60001F46241900986D41401C00903428E1DD48
:105A7000F91930467041091BA84103D20022D243D4
:105A8000134601E00022134601980105381C7141BC
:105A9000FFF751FFB6E70000064C0125064E05E072
:105AA000E36807CC2B430C3C98471034B442F7D33F
:105AB000FFF70AFB50C5000870C5000870B58C18C8
:105AC0000578401C6B075B0F01D10378401C2A113D
:105AD00006D10278401C03E006780E70401C491C79
:105AE0005B1EF9D12B0705D40023521E0DD40B7079
:105AF000491CFAE70378401CCB1A921C03E01D787E
:105B00000D70491C5B1C521EF9D5A142D8D3002050
:105B100070BD000038B50446064805490068FFF727
:105B2000E7FA604300E0401E00900028FBD138BD3A
:105B300040420F009C010020F8B5044600688168CF
:105B40008907890F012902D10168C90722D181681B
:105B5000114A10261140012500290ED181682943E0
:105B600081600120FFF7D6FF01F046F807460CE000
:105B700001F042F8C01B0A2807D9606D3043606508
:105B8000A06D2843A0650120F8BD20680068C043CF
:105B9000C007EDD10020F8BD1700008010B501202E
:105BA00005F064FD0A4C1328A0700AD0E01C02F036
:105BB00087FCE078A070332806D006490020C8870B
:105BC00010BD05F08BFD10BD02F04CFC10BD0000B7
:105BD00000000020000E00201FB50B4800900B486D
:105BE00001900B4802900B48039069460A4804F064
:105BF0005DFF0A4A08481146083904F045FE00F0E6
:105C00006FFA002004B010BD5DC3000839C300085E
:105C100099C3000897C30008A801002028000020AD
:105C200010B500231A4603E0845CE3189BB2521CB3
:105C30008A42F9D3D84380B210BD000010B50348A2
:105C400000F096FD024800F093FD10BDB017002053
:105C50006817002030B5446C1C252C400125A54058
:105C6000046C6560046863608368102B036803D06C
:105C700099600068C26030BD9A600068C16030BD44
:105C80001449012048720A4602205E3250720320F5
:105C90003C3A507204200E3A50720F480D4B007877
:105CA000087022310870203108770C495A1C087896
:105CB00058714978997123331871597120331877C5
:105CC0005977107551751A461E3210755175107638
:105CD0005176704700120020560100207801002004
:105CE00010B503F0FDFC202003F0B8FD012005F005
:105CF00047F9002003F0B2FD044804F0E5FF044832
:105D000005F094FA002005F0C9FA10BD1801002032
:105D100083800000F8B503F0AFFD052001210007E6
:105D200000F056FF0025144C002800D06560134E8B
:105D30000221304600F04CFF002815D101202070D0
:105D40000F48808F00280ED00127BF02002239465D
:105D5000304600F04AFF0A2004F006FD01223946D1
:105D6000304600F042FF6560012000F069FE02202D
:105D700000F066FEF8BD000088010020000400501D
:105D8000000E00207047000010B5084900224A614B
:105D900007494B684C1523434B604B680824234349
:105DA0004B60C009C001026010BD0000F817002060
:105DB000002002407FB500250C460646039500F002
:105DC0000FFEE009029003A901960095684600F0D5
:105DD0009FFD002804D000F0D7FD002004B070BD66
:105DE00000F0D2FD0120F9E710B5002302E0C45C09
:105DF000CC545B1C9342FAD310BD000010B5214A6D
:105E000000219069C305204804D541690223194344
:105E10004161911593699B0505D54369012423438D
:105E200043616302194393695B0505D543690824FF
:105E300023434361E301194393691B0505D5436976
:105E40000424234343616302194393699B0405D5EA
:105E500043691024234343616302194393699B03FD
:105E600004D5446920231C43446119439369DB032F
:105E700005D54369402423434361A0020143916156
:105E800010BD000000200240F817002070B5054644
:105E900000F0B2FE0646184C0AE0681C08D0002D3F
:105EA00004D000F0A9FE801BA84201D9032070BDD8
:105EB000A069C007F1D1A069800701D50220A061C7
:105EC000A069C00511D4A06980050ED4A069400561
:105ED0000BD4A069000508D4A069800405D4A0698A
:105EE000800302D4A069C00303D5FFF787FF012018
:105EF00070BD002070BD000000200240F8B51746BC
:105F0000002605460C4600F06BFD09E029460220FC
:105F1000226800F047FD002804D1241D2D1D361DE8
:105F2000BE42F3D300F030FDBE4201D20020F8BDE6
:105F30000120F8BD10B5084902460020054B4979FB
:105F400005E044001C5B944203D0401CC0B2884270
:105F5000F7D310BDA41300208800002010B500F076
:105F60003CFE10BD10B5094801F05CF880B2FFF7A7
:105F7000A7FB074A074BFFF787FA0022064BFFF7FC
:105F8000EBFAFFF7E3FB80B210BD00001C16002007
:105F9000F853E3A59B843E4000408F4070B5002439
:105FA000204603F01DF847494748A200641CE4B2AC
:105FB0008150142CF9D3464944480A79027549792D
:105FC000417544490A780276497841763F4905206F
:105FD000133148720A2005F019F97D20400105F0BF
:105FE0002FF93A49002213310C2005F0F9F900216C
:105FF0000C2005F007FA384801F014F8344C01255C
:10600000223C2085AD0309E0334801F00BF880B253
:106010002085E18EFF392D39884206DBE18E80B282
:106020008842F1D349198842EED8022005F03EF9A2
:10603000002002F0D5FF294D00210F2005F066F861
:1060400028422064F8D0206C411C38D0400435D55B
:106050008122D20100210F2005F097F900211020A4
:1060600005F054F841061948490E0022C73005F0E2
:1060700083F8164DC735687A05281FD102221549C5
:10608000681DFFF79FF8002818D11148AE7C667193
:106090000422691C3630FFF771F82946133108468F
:1060A00072000D466930FFF769F8607929464200B1
:1060B00005484838FFF762F80320207070BD04F0EF
:1060C00073F90000FFFF010004140020611200209A
:1060D000AA000020780100201C16002000D02724F0
:1060E00010B5144C1448224610321146083904F0F9
:1060F000CBFB0022114BE168A068FFF72DFA104A94
:10610000104B05F0BBFB00220F4BFFF7B5F9002247
:106110000E4BFFF7B9F9FFF773FB2060002213461F
:10612000E168A068FFF744FB01D0206810BD0020A3
:10613000206010BD18000020A801002000AA8F4098
:106140006C45D9CC955BC83F0000F03F40A5E540C9
:1061500010B5084800F096FA0A21064800F032FA15
:10616000044800F01DF9800503D5024800F01AF933
:1061700080B210BDC0150020F8B52F4D00220121BE
:10618000284600F032FDFFF7E3FFFFF77EFA2B4EC3
:106190003146FFF77DF82A4C0122A06011462846BF
:1061A00000F023FD2749A068002588423EDB2078C7
:1061B000254F002815D02570FFF7CAFFFFF765FAB5
:1061C0003146FFF765F8A060FFF7DEFA00223B4694
:1061D000FFF74CF900221D4BFFF756F9FFF710FBB4
:1061E0006060A068FFF7D0FA00223B46FFF73EF957
:1061F000174A184BFFF748F906460F466068FFF745
:10620000C3FA134A144B5242FFF73EF932463B465B
:10621000FFF788F8FFF7F4FA10496060884201DD63
:10622000616004E0FF21C905C84200D36560606871
:10623000FFF754FAC0B2F8BD0004005000401B4400
:10624000600000200000604000000C4000E064405E
:106250003333333333B33040CCCCEC3F0000C8424F
:10626000F8B5054604464035287C0026012808D0AC
:1062700001202874206881688907890F01290ED1BF
:1062800001E00220F8BD0168C90708D0606D202137
:10629000084360650126002028743046F8BD616D12
:1062A000FF2201329143022211436165C1688907CF
:1062B000890F0091C16889088900C16020688168E0
:1062C00092071143816000F097FC07460EE000F052
:1062D00093FCC01B0A2809D9606D02218843102154
:1062E00008436065002028740120F8BD206880689C
:1062F0000028ECDB2068C168009A1143C160606D22
:1063000080088000401C6065C5E70000F8B50646BF
:106310000D464036317C01290DD0012131740168D0
:106320008A68520709D5416D20221143416500203A
:1063300030740120F8BD0220F8BD174B6A68D805FB
:1063400047109A42154C8A6A2B6812D05B035B0B8C
:106350001A438A622968490305D5A1680143A160EF
:106360000A20FFF7D7FB2868800312D5A0683843BE
:106370000EE05B035B0B9A438A622968490302D5EE
:10638000A1688143A1602868800302D5A068B84352
:10639000A06000203074F8BD01100000002701400B
:1063A000406D70470068006C7047000070B50400D5
:1063B00006D0606D264600254036002802D006E053
:1063C000012070BDA5653574204600F0D3F8606DDE
:1063D000C00603D421688868400705D5606D102188
:1063E000084360653574EBE7606DFF22013290432E
:1063F00002221043606588688207920F5B48012A79
:1064000002D10A68D2072BD1032362689B079A4204
:1064100005D05B429A4202D05B009A4209D10A69D8
:10642000920092080A6121680A6963681A430A6146
:106430000CE00A69920092080A6181680F229204B6
:106440009143816081686268114381602168CA68F4
:1064500018239A43CA602168CA68A3681A43CA60AD
:10646000816801225206914381608168A28E5206A2
:106470001143816020688168C90004D481680122C9
:106480001207114381602068C168394A1140C16018
:106490002069E168022825D00020014320462030F1
:1064A0000278037B52035B001A431143226B1143B2
:1064B000A26992031143E269D20311432268D368AF
:1064C0001943D160616A0A46FF3AC23A05D0A26A0E
:1064D00011432268D3681943D16042780121012A0F
:1064E00002D00BE00420D8E70078002823D0606DAC
:1064F000202210436065A06D0843A065E06B012871
:1065000020681FD00169C90703D001694908490003
:10651000016120684169C908C90041612068416979
:10652000A26B11434161A565606D80088000401C2D
:106530006065002070BD2068C26801231B041A43F7
:10654000C260DBE70269FF239B009A430261206877
:106550000269236CA66C1A43636C33431A430261CD
:10656000206802690A430261D3E700000027014066
:106570001902FEFF10B586B0044614216846FEF7E6
:1065800016FE0E492068884216D10D48416B42150F
:1065900011434163C16A01221143C162C06A694665
:1065A00010400590022000900320019000200290EE
:1065B0000520000700F050FA06B010BD002401408D
:1065C00000100240F8B504464069254640350E46A5
:1065D00008280BD02068C068C00709D0606D202152
:1065E00008436065002028740120F8BD082700E0FA
:1065F0000C2700F001FB009011E0701C0FD0002E62
:1066000005D000F0F9FA0099401AB04207D9606D40
:10661000042108436065002028740320F8BD206829
:1066200000683842E9D0606D012149020843606585
:106630002068C16809058A0F0C21002A1BD120227D
:10664000125D002A17D10268120714D58268530719
:106650000122002B08DB43688B434360606D13020B
:1066600098431043606506E0606D20231843606521
:10667000A06D1043A065A069002801D120680160C9
:106680000020F8BD70B504462168002089684907DC
:1066900021D425464035297C01291CD001212974AB
:1066A000E169012904D02046FFF746FA002811D1FC
:1066B000616D0A4A1140FF220132114361650021D8
:1066C000A165297422681C21116021688A6804234D
:1066D0001A438A6070BD022070BD0000FEF1FFFF0A
:1066E00030B5014620314A790023022A04D0042221
:1066F000C2630B71012030BD026814680E25AC43E3
:10670000146002681468640864001460446C1C22FD
:10671000144001221546006CA54045604A71184698
:106720000B7130BD70B50024014620314A79022A30
:1067300003D00421C163012418E0026813680E2508
:10674000AB431360026813685B085B001360436C23
:106750001C221340012215469D40036C5D604A7166
:1067600000220A71816B002900D08847204670BD45
:10677000F0B4016C0D6801680C68466C1C2304229F
:106780001E401746B7402F420ED067070CD50C6845
:10679000A40602D40C6894430C60416C19408A40F2
:1067A000016C4A60016B1AE00227B74002462F4095
:1067B0002032002F17D0A70715D50C68A40605D4E2
:1067C0000C680A25AC430C6001215171446C022114
:1067D0001C40036CA140596000211171C16A00295D
:1067E00018D0F0BC08470827B7402F4212D0240722
:1067F00010D50C680E25AC430C60446C01211C4084
:106800000B46A340046C6360C16351710021117198
:10681000416BE4E7F0BC704770B504003CD01F4802
:10682000256814212818FEF763FC800060641C486A
:10683000206402212046203002464171296819480F
:10684000E3680140A068666918432369334318432D
:10685000A3691843E3691843236A1843084328606F
:106860000121A0688903884210D00D488030836AD6
:10687000656C1C210D400F26AE40B3438362656CEE
:1068800063680D40816AAB400B4383620020E06384
:1068900001215171107170BD012070BDF8FFFDBF65
:1068A000000002400F80FFFFF8B504468C46203000
:1068B00001790025012909D00126067141790027B7
:1068C000012905D0077102252846F8BD0220F8BD30
:1068D00002214171E76320680168490849000160AD
:1068E00061462046FFF7B6F9206B00282068016852
:1068F00001D00E2205E00422914301602068016866
:106900000A22114301602068016831430160DBE71E
:10691000F8B51A4E0546307C0F46012807D00120F5
:1069200030741748FFF7B2FA010002D021E00220CC
:10693000F8BD0020C04338606C6814E02046FFF7C3
:1069400023FA0F48FFF7A2FA01460E4842680823CF
:106950009A434260426843159A434260002901D03D
:106960003C6006E08034A8686A68C0018018A042D4
:10697000E4D8002030740846F8BD0000F817002065
:1069800050C3000000200240054841680222114324
:1069900041604168012211434160002070470000BE
:1069A00000200240F8B50C4C1646207C0F4601280A
:1069B00008D0012020740948FFF768FA0025002854
:1069C00002D006E00220F8BD65613E600348FFF793
:1069D0005DFA2574F8BD0000F817002050C30000D0
:1069E00011484168C9070BD0EFF3108172B60F4A06
:1069F000C2600F4AC26081F310884168C9070ED196
:106A0000416889070DD5EFF3108172B6094A02611A
:106A1000094A026181F310884068800701D501208E
:106A2000704700207047000000200240EFCDAB8986
:106A300005040302BFAE9D8C1615141370470000A9
:106A400010B504494A69024202D04861FFF7F6FFD7
:106A500010BD000000040140FCB500230124A2E0A9
:106A600027462A469F403A406FD04D68012D05D0F9
:106A7000022D03D0112D01D0122D16D185680326C9
:106A8000AC465D00AE46AE406546B543AC46CE680A
:106A90007546AE4065462E43866046680D79BE4316
:106AA000ED06ED0F9D4035434560C6685F00032548
:106AB000BD40AE46AE4335468E68BE402E43C660EE
:106AC0004E68022E01D0122E14D1DE08B600361800
:106AD0000196366A5D07B446EE0E0F25B540009666
:106AE0006646AE43B4460D69009EB54066462E43E9
:106AF000019D2E6206687546AE430D79AD07AD0F58
:106B0000BD40354305604D68ED004BD5294D6E6B9A
:106B100026436E639E08284DB6007519AC46AD68D5
:106B20009E07360F0F27B740BD4305273F07B842E2
:106B300001D1002715E0214FB84201D1012710E013
:106B40001F4FB84202D102270BE02BE01D4FB84285
:106B500001D1032705E01C4FB84201D1052700E011
:106B60000627B7402F436546AF60184D2E684F6823
:106B70009643FF0300D516432E606E684F68964318
:106B8000BF0300D516436E60AE684F689643FF02A0
:106B900000D51643AE60EE684F689643BF0200D53D
:106BA0001643EE605B1C0A681546DA4000D057E7D2
:106BB000FCBD000000100240000001400004005035
:106BC00000080050000C0050001C00500004014060
:106BD0000069084000D001207047426913460B400D
:106BE0001B0491430B4383617047002A01D08161EC
:106BF000704781627047000001488068704700005C
:106C000090010020024881680278891881607047ED
:106C10009001002010B5084800240168402211436B
:106C20000160204600F00AF8002801D0012401E0AC
:106C300000F042FA204610BD0020024070B5044624
:106C40000D4D7D202978C000FEF752FA01460B4811
:106C50000068FEF74DFA00F02BFF002809D1042C44
:106C600007D200222146401E00F04EFA00206C6040
:106C700070BD012070BD0000900100209C0100202B
:106C800070477047F8B502F0F7FD604C0120E070E6
:106C9000208AFEF7FAFC01467F20C005FEF7F8FACD
:106CA0005B4D06462968FEF79AFA28600120A16A22
:106CB000C005814201DA084603E03046FEF7E4FAF7
:106CC000A062FF21C9050025C84200D3A5626078F3
:106CD00000280BD102214F48FFF77AFF02004E49EE
:106CE0004E4817D00022FFF780FFE5620221494895
:106CF000FFF76EFF4A4E002855D0E562B08AFEF7D6
:106D0000C4FC434F3968FEF797FD5FD24549012027
:106D100008705DE00122D1034048FFF766FF208A3A
:106D2000FEF7B3FC01467F20C005FEF7B1FAE16A29
:106D3000FEF755FA3C49E0628842D7DD3848012722
:106D4000F926403000900A213046FEF7D1F900299B
:106D500003D131493148FFF701F902212D48FFF7EE
:106D600037FF002801D0002701E0002F12D10221B7
:106D70002848FFF72DFF00280CD104F047FD0099AB
:106D80000120888005F09EFA642003F0EDFC28497C
:106D90002648C8600A2003F0E7FC3046761EF6B2AB
:106DA0000028D0D1A2E7208AFEF76FFC01467F20A1
:106DB000C005FEF76DFAE16AFEF711FA1D49E062BF
:106DC00088429BDB1A491948C86097E71548057047
:106DD000708F401EFEF74EFC3968FEF72DFD06D879
:106DE0002079002803D014490120087001E01248DE
:106DF0000570708FFEF749FC3968FEF71DFD04D25F
:106E00002079002801D004F0F5FBF8BD54010020E2
:106E10008C010020000400500080000000000050A1
:106E2000000E00208E000020000040400400FA0503
:106E300000ED00E00000A0409E000020704770B50B
:106E4000040010D0022025462035A873204601F00A
:106E50008BFBA87B032805D0204600F0B9F8002062
:106E6000A873687370BD012070BD7047704710B57E
:106E7000044600680168C943C90708D18168C9434D
:106E8000C90704D1012141602046FFF7FBFE2068BD
:106E90000168C943890708D48168C943890704D4B4
:106EA000022141602046FFF7EBFE20680168C943DC
:106EB000490708D48168C943490704D404214160C3
:106EC000204600F0F7F820680168C943090708D494
:106ED0008168C943090704D4082141602046FFF7AF
:106EE000ADFF20680168C943C90608D48168C94359
:106EF000C90604D4102141602046FFF7C2FE206875
:106F00000168C943890608D48168C943890604D445
:106F1000202141602046FFF7A9FF20680168C9438E
:106F2000490608D48168C943490604D44021416018
:106F30002046FFF79AFF10BDF8B5040005D025469E
:106F40002035A87B002802D006E00120F8BD0020F3
:106F50006873204600F04EF80220A8732068C268CB
:106F600084466368012B01D106208243164861697B
:106F7000814202D0072040038243002B01D1D82058
:106F800082431248A668024018463043676A266A60
:106F90003E433043A66A30431043002B02D0012BFE
:106FA00004D005E02369E2691A4300E0E268104377
:106FB000054A914202D0A269114308436146C86064
:106FC0000120A8730020F8BDFFFF0000F8F119FFB1
:106FD00010B500680549884207D10548816B490012
:106FE000490881630D2000F073F810BD007C00405B
:106FF0000010024010B50068084988420CD10848CA
:10700000816BC20411438163002201210D2000F035
:107010007BF80D2000F06CF810BD0000007C0040F3
:10702000001002400068C06970470000F8B50446CF
:107030000220254620351746A8731D480268C30460
:107040001A4302602068C2689B121A43C26020681B
:1070500002690126324302612268102050602068D4
:1070600081611021204601F0EFFA03281FD021682A
:1070700008204860206847610821204601F0E4FAB2
:10708000032814D0204601F06FFAA87B03280ED005
:107090002068816831438160206801693143016162
:1070A00020680169042211430161AE730020F8BD1C
:1070B00000040140704700000448416B0122114365
:1070C0004163816B020411438163704700100240E9
:1070D000002809DBC106C90E012088400349086069
:1070E000BFF34F8FBFF36F8F7047000080E100E068
:1070F000002805DBC106C90E01208840014908604F
:107100007047000000E100E010B503F02BF910BD5E
:1071100002494A6882434A6070470000007000409C
:1071200002480168821511430160704700700040F9
:1071300002494A6802434A607047000000700040FC
:1071400005480168022211430160044801690422D4
:107150001143016130BF70470070004000ED00E056
:10716000F0B5154A1368154D54152D6A2340ED07E7
:10717000ED0F002B04D0002D02D01668A643166038
:107180001668B608B600064316600D48076904265F
:107190003743076101290DD040BF20BF20BF0169DF
:1071A000B1430161002B04D0002D02D010682043B0
:1071B0001060F0BD30BFF2E70070004000000140F9
:1071C00000ED00E0F8B5044600780027534D800636
:1071D00071D5524E403EB06BC00004D4B06BA905CF
:1071E0000843B06301274E480168C90511D40168FE
:1071F000821511430160FFF7FFFC009005E0FFF7E7
:10720000FBFC0099401A642837D845480068C0053F
:10721000F5D532680321090560680A4001409142B2
:1072200008D08103890F032904D13168890301D56E
:107230000120F8BD2A69032109040A4022D0084030
:1072400090421FD0207880061CD528692A6988437F
:107250000121C9040A432A612A698A432A612861F3
:10726000C0050FD5FFF7C8FC009008E0FFF7C4FC8D
:107270000099411A2B48814201D90320F8BD2869A1
:107280008005F3D561688803800F032805D1326833
:107290000005824301400A43326028690322616885
:1072A0001204114008432861002F04D0B16B012063
:1072B00000078143B1632078C00705D0E868A16862
:1072C000800880000843E8602078800705D5E868DA
:1072D0000C218843E1680843E8602078400706D520
:1072E000E86803218902884321690843E86020781F
:1072F000000706D5E868032109038843616908434C
:10730000E8602078000606D5E868032189048843F0
:10731000A1690843E8600020F8BD00004010024069
:107320000070004088130000F8B50E46050038D004
:107330005E480068C007C00FB04214D25B4C2068A2
:107340004008400030432060FFF756FC074605E048
:10735000FFF752FCC11B564881427AD82068C0070B
:10736000C00FB042F4D12878524C800705D5E068B0
:10737000F0218843A9680843E0602878C00752D00C
:107380006868022806D0032807D0216801280AD09F
:10739000890504E02168890301E021688901002949
:1073A00003DB0120F8BD4907F9E7E1688908890096
:1073B0000143E160FFF720FC0746686802280AD015
:1073C000032814D001281ED029E0FFF715FCC11BAB
:1073D000374881423DD8E0680007800F0228F4D189
:1073E00021E0FFF709FCC11B3148814231D8E06838
:1073F0000007800F0328F4D115E0FFF7FDFBC11B48
:107400002B48814225D8E0680007800F0128F4D17D
:1074100009E0FFF7F1FBC11B2548814219D8E0685C
:107420000007800FF5D121480168C907C90FB14293
:1074300017D901684908490031430160FFF7DCFBB7
:10744000074608E005E0FFF7D7FBC11B184881425B
:1074500001D90320F8BD15480068C007C00FB0422D
:10746000F1D12878400706D5E06807210902884352
:10747000E9680843E0602878000707D5E06807213D
:10748000C90288432969C9000843E06000F03AF85E
:10749000E168094A0906090F515CC84007490860BC
:1074A00007480068FFF7CAFBF8BD00000020024053
:1074B00088130000001002409EC400089C010020B8
:1074C00094010020044805490068C968044A490538
:1074D000490F515CC84070479C01002000100240D9
:1074E000B7C40008044805490068C968044A89040B
:1074F000490F515CC84070479C01002000100240B9
:10750000B7C4000870B51A4AD3681A490C2018404D
:107510008D0004280CD04E00082810D00C2810D064
:1075200050680004410F0120C003491C884070BD11
:107530001068C00601D5084670BD284670BD3046AB
:1075400070BD98020C4C000F205C1B029C0FD3688E
:10755000641CDB0301D5314603E01268D20600D477
:10756000294602F0C4FE22460023FDF7D7FD70BD78
:107570000010024000093D00AEC40008FEB5050041
:107580007ED0FE4CE7680C20E6680740012000042E
:1075900006402878C00747D0082F05D00C2F0AD105
:1075A00001200004864206D1206880033CD568682B
:1075B0000028E5D038E0012069680004814203D149
:1075C00021680143216011E0052301221B0492047C
:1075D0009942216802D111432160F1E78143216082
:1075E000216801400091206890432060686800286D
:1075F0000DD0FFF701FB009005E0FFF7FDFA0099C1
:10760000401A64287BD820688003F6D50CE0FFF789
:10761000F3FA009005E0FFF7EFFA0099401A6428AA
:10762000F0D820688003F6D42878800756D509233F
:10763000E868042F0DD00C2F01D1002E09D00028AE
:107640003CD02168994301432160FFF7D5FA0646F3
:1076500028E02168490701D5002891D061681F22E0
:10766000120291432A691202114361602168994311
:1076700001432160FFF746FFE16809060A0F00E0B9
:107680008BE1BF49895CC840BE490860BE480068BC
:10769000FFF7D4FA002873D120E0FFF7ADFA801B82
:1076A0000228AFD820684007F7D560681F2109027B
:1076B000884329690902084360600FE02068400898
:1076C00040002060FFF798FA064604E0FFF794FABE
:1076D000801B022896D820684007F7D42878C00677
:1076E00060D5002F0CD0A86900284AD02068FF215F
:1076F000013108432060FFF77FFA06462EE0C1E023
:107700002068800502D5A8690028A6D060680721F6
:1077100049038843296A084360606068297F000242
:10772000000A090608436060286A410B0120C00373
:10773000491C8840E16809060A0F9149895CC840E4
:107740009049086090480068FFF778FA002817D140
:1077500028E0FFF751FA801B0228A2D82068800594
:10776000F7D56068072149038843296A08436060A8
:107770006068297F0002000A09060843606011E082
:10778000E2E02168FF20013081432160FFF734FAF5
:10779000064604E0FFF730FA801B022872D8206802
:1077A0008005F7D42878794E000724D56869002829
:1077B000306910D0012108433061FFF71DFA0090B5
:1077C00005E0FFF719FA0099401A02285AD83069E3
:1077D0008007F6D50FE0400840003061FFF70CFA53
:1077E000009005E0FFF708FA0099401A022849D8EE
:1077F00030698007F6D42878400766D500200290CB
:10780000A06BC00006D4A06B012109070843A06348
:10781000012002905E480168C90511D401688215F3
:1078200011430160FFF7E8F9009005E0FFF7E4F984
:107830000099401A642825D855480068C005F5D538
:10784000FF20AA680130824203D1316901433161CE
:1078500011E001218902002A07D005231B029A4268
:1078600003D132690A433261EFE732698243326100
:10787000306988433061A868002810D0FFF7BCF950
:10788000009008E05FE0FFF7B7F901460098091A99
:107890004048814257D830698005F4D50DE0FFF7A4
:1078A000ABF9009006E0FFF7A7F90099411A3948B3
:1078B000814248D830698005F5D40298002804D068
:1078C000A06B012109078843A063686A002866D07D
:1078D0000C2F3ED0012636060228206805D0B04382
:1078E0002060FFF789F905462FE0B0432060FFF7DD
:1078F00083F9074604E0FFF77FF9C01B022822D86E
:1079000020688001F7D4E96AA86AE2680843296B15
:10791000FD231B049A4311430843E0602068304371
:107920002060FFF769F9054604E0FFF765F9401BA1
:10793000022808D820688001F7D530E0FFF75CF90D
:10794000401B022801D90320FEBD20688001F5D428
:1079500025E00128F8D0E06801210904AA6A014065
:1079600091421AD10F218904EA6A0140914214D14F
:10797000032189050840296B88420DE00010024070
:107980009EC400089C010020940100204010024089
:10799000007000408813000001D00120FEBD0020CF
:1079A000FEBDF8B504000ED0FF27606A053700253C
:1079B00000280AD02561656126464036A562707CA4
:1079C000002807D00AE00120F8BD6068B842F3D073
:1079D000E561F1E73574204600F03EF8022171744C
:1079E0002068026840239A4302602123A2686068ED
:1079F0009B021A4038401043E3688A021340184340
:107A000023690B40217D1843C907C90F0843A169A9
:107A1000931019400843E169382319400843216A4B
:107A2000802319400843A16A930019400843216844
:107A30000860A0690421000C0840616A1023194005
:107A40000843216848602068C1699143C161656548
:107A5000012070740020F8BD10B586B004461421D2
:107A60006846FDF7A4FB10492068884219D10F48E9
:107A7000416B821411434163C16A01221143C16207
:107A8000C06A002110400590E02000900220019083
:107A90000320039002910491052069460007FEF738
:107AA000DBFF06B010BD00000030014000100240B6
:107AB000094910B5401E884201D9012010BD074C6C
:107AC00060610321081F02F04DFC0020A061072027
:107AD0002061002010BD0000FFFFFF0000E000E07B
:107AE00070B505462C4602202034002908D0042910
:107AF0000BD008290ED0627F012A10D0012070BD62
:107B0000A27E012AFAD1A0760AE0E27E012AF5D10E
:107B1000E07605E0227F012AF0D1207700E060774F
:107B20000122286801F01EFF012228689207012126
:107B3000904205D0074A904202D0074A904204D1B1
:107B400082685207520F062A02D002680A43026076
:107B5000002070BD000801400014014070B50446CB
:107B60000D460068002201F0FDFE2068016A0C4A03
:107B7000114203D101684908490001600120203405
:107B8000002D06D0042D06D0082D06D060770020E9
:107B900070BDA076FBE7E076F9E72077F7E7000015
:107BA000111100007047704770470000F8B5026877
:107BB0000446D06911689668814B05461D40202314
:107BC000002D6CD0F7077F4DFF0FBC460D402F43B3
:107BD00079D02546C7078035002F06D0CF0504D5BC
:107BE000012717622A683A432A60820708D5F207FC
:107BF00006D0276802223A622A6804273A432A609C
:107C0000420708D5F20706D02668042232622A68A5
:107C1000022632432A6002070AD50A461A406646FF
:107C2000324305D02668082232622E6816432E6041
:107C3000020508D54A0106D501222668D202326221
:107C40002A681A432A602A68002A30D0800606D59E
:107C5000880604D5616E002901D02046884728682F
:107C600021688968490602D42821084225D0204687
:107C700002F089F820688168490619D58268402198
:107C80008A438260206F002812D04F498163206FA1
:107C9000FEF748FD00280AD0206F816B06E08506BC
:107CA00011D58D060FD5616E77E020468847F8BD67
:107CB0002046FFF779FFF8BD05E02046FFF774FF87
:107CC00000202860F7E7256E012D56D1C50654D552
:107CD000CD0652D5102616622068816825464906D1
:107CE000403500292ADA226F116849680904090C15
:107CF000E1D02F8B8F42DED969831168096889062C
:107D000017D40168320191430160206881684908F5
:107D10004900816020688168402291438160E36767
:107D20000020206620680168B1430160206FFEF7E3
:107D3000D7FC288B698B401A81B21AE0298B6A8B99
:107D4000891A6A8B89B2002AB5D00029B3D002689B
:107D5000FF252135AA43026020688268520852003C
:107D60008260E36700202066606620680268B24394
:107D700002602046FFF716FF9DE7C50208D5750291
:107D800006D50120000510622046FFF70CFF92E7A0
:107D9000050605D50D0603D5A16E002985D18AE714
:107DA000400688D5480686D5116820464024A14360
:107DB000116083670021816600F043F97BE70000D2
:107DC0000F08000020010004AD9C000810B504005D
:107DD00003D0A06F002802D007E0012010BD0021D1
:107DE00074200155204600F027F82420A067206861
:107DF0000168490849000160204602F017F801288F
:107E0000ECD0606A002802D0204601F039FE2068DC
:107E100041680922D20291434160206881682A2288
:107E2000914381602068016801221143016020466E
:107E300001F08CFE10BD0000F0B587B0064614219D
:107E40006846FDF7B4F92C493068884251D12B4877
:107E5000416B0122920311434163C16A0122114324
:107E6000C162C06A002510400590032040020090C6
:107E70000220032701A9A1C104200490052069461E
:107E80000007FEF7E9FD1F4C1D48A560E56081C4B1
:107E90008027E560A7602020256160610002A06165
:107EA0001848083CFEF7B8FC002801D0FDF76AFF2F
:107EB0003467A662144C124821461438206003200F
:107EC000606010200831A1C16561A561E5612046AF
:107ED0002562FEF7A1FC002801D0FDF753FFF466F0
:107EE000002201211B20A662FFF70EF91B20FFF7DD
:107EF000FFF807B0F0BD000000380140001002405C
:107F00003000024068170020B017002070B5C36F22
:107F1000202B27D100290BD0002A09D00124836807
:107F20002403A34206D10369002B03D1CB0701D060
:107F3000012070BD034660331C7D012C12D001244A
:107F40001C7500230366084C0368A34207D05C68D5
:107F5000240204D51C680125AD062C431C6002F0E8
:107F600065F870BD022070BD004800407047704742
:107F7000FFB50446806F83B017460D4620285ED1BA
:107F8000002D0AD0002F08D0A168C001814207D17E
:107F90002069002804D1E80702D0012007B0F0BD15
:107FA000204660300090007D012848D000980121D3
:107FB00001750020802108512120A067FEF71CFEDA
:107FC000264640360190378277820120A16800035F
:107FD000814202D12069002805D02F460025009952
:107FE0000020087511E00027F9E7002280212046D3
:107FF00002F062F8002815D1002F15D021683878DA
:1080000088627F1C708A401E7082708A019B0028E3
:1080100006980090E9D100224021204602F04CF859
:10802000002808D00320B9E728882168C005C00DC2
:108030008862AD1CE6E72020A0670020AEE70220A2
:10804000ACE77047034D044C04A002F02FF9E56043
:10805000FAE700000400FA0500ED00E048617264F0
:108060004661756C745F48616E646C65722E0D0AB2
:108070000000000070B586B014216846FDF797F83F
:1080800001240B480C4EC4800A48A50244832246B2
:1080900029463046FEF7A9FD002102910391009583
:1080A000019469463046FEF7D7FC06B070BD00006B
:1080B000400E0020540100200004005010B505249B
:1080C0002407002204212046FEF78FFD002208210C
:1080D0002046FEF78AFD0A2002F04DFB0122042112
:1080E0002046FEF782FD0A2002F045FB0022042113
:1080F0002046FEF77AFD10BD10B5052424070022A6
:1081000004212046FEF771FD012208212046FEF7DA
:108110006CFD0A2002F02FFB012204212046FEF70D
:1081200064FD0A2002F027FB002204212046FEF70E
:108130005CFD10BDF8B50024052607462546360728
:10814000002204213046FEF750FD0A2002F013FB06
:10815000012204213046FEF748FD6006040E082186
:108160003046FEF735FD002801D0641CE4B205203E
:1081700002F001FB6D1CEDB2082DE1D3002F03D0FE
:10818000FFF79CFF2046F8BDFFF7B6FFFAE770B592
:10819000052605463607002204213046FEF725FD58
:1081A0000024E80901D0012200E000220821304625
:1081B000FEF71BFD6806050E0A2002F0DCFA01221C
:1081C00004213046FEF711FD0A2002F0D4FA002205
:1081D00004213046FEF709FD0A2002F0CCFA641CA7
:1081E000E4B2082CDDD370BD10B5052424070122AC
:1081F00008212046FEF7F9FC012204212046FEF763
:10820000F4FC002208212046FEF7EFFC0A2002F0D1
:10821000B2FA002204212046FEF7E7FC10BD10B59B
:1082200005242407002204212046FEF7DEFC00225C
:1082300008212046FEF7D9FC0A2002F09CFA012210
:1082400004212046FEF7D1FC012208212046FEF73A
:10825000CCFC0A2002F08FFA10BD70B505252D0761
:108260000024012208212846FEF7BFFC062002F068
:1082700082FA012204212846FEF7B7FC062002F00C
:108280007AFA07E0641CE4B2FA2C03D9FFF7C7FFBF
:10829000012070BD08212846FEF79AFC0028F1D184
:1082A000002204212846FEF7A0FC002070BD00003B
:1082B000F8B501F07DFC01F0ADFC5B480068C069D9
:1082C000FDF750FE594C5A49A082898F594E00251E
:1082D000002931D0A26A730357499A4202DB022275
:1082E0000A7000E00D700A7801218902002A05D089
:1082F000012A0ED0022A10D0032A1DD1608B01283A
:108300002ED0022818D1484808214038FFF726FC13
:1083100012E0FF22F5329042F0D2608B01281DD08E
:10832000022804D008E03046FEF75FFC04E03E4837
:1083300008214038FFF7D4FBFDF71EFF2070012114
:10834000C9023046FEF744FC0127FF0300282DD068
:108350003A480560A079002804D007E00022E2E74F
:108360000122E0E70120A07101F008FF80213046E2
:10837000FEF72EFC002806D0002208213046FEF72A
:1083800034FC012205E0012208213046FEF72DFCD5
:108390000022052039460007FEF727FC244C284E12
:1083A0004034A08C274F012803D01CE0A571002287
:1083B000EAE725486946088072B680212348FDF720
:1083C000F9FC002804D0022269462048FDF796FDFA
:1083D00062B61FA001F06AFFA58403F073FF64205A
:1083E00002F0C2F9FE60608C012808D11048658453
:1083F000058003F067FF642002F0B6F9FE60208C70
:10840000012806D1258403F05DFF642002F0ACF959
:10841000FE600748124A0188914202D1C0880028B4
:1084200000D1FE60F8BD0000E416002054010020D9
:10843000000E0020000400509C0000208C01002051
:108440000400FA0500ED00E0AAAA0000384A00087E
:10845000BDF8C8EBC9FDBCB6C4A3CABD0D0A000077
:10846000AA55000010B53721202000F070F8032134
:10847000212000F06CF84021222000F068F808214B
:10848000232000F064F8AA21302000F060F80A48A8
:1084900001210187322000F05AF80121332000F039
:1084A00056F85F21202000F052F8044800F008F848
:1084B0000A2002F060F910BD000E00200300002029
:1084C00010B501460F2000F021F8002800D001204F
:1084D00010BD10B50446FFF787FE3220FFF757FEA8
:1084E000FFF7BBFEE0B2FFF752FEFFF7B6FEFFF765
:1084F0007BFE3320FFF74BFEFFF7AFFE0020FFF7B8
:1085000019FE0446FFF78BFE204610BD10B50C4641
:10851000FFF7DFFF2070012010BD70B50D46044647
:10852000FFF762FE3220FFF732FEFFF796FEE0B261
:10853000FFF72DFEFFF791FE2846FFF728FEFFF715
:108540008CFEFFF76CFE0A2002F015F970BD10B525
:10855000FFF7E3FF012010BD10B50248FEF787FCCE
:1085600010BD00001C160020FEB50446002772B6A0
:10857000334A01688B1804D13248C768032080044D
:10858000074088680190C868009048698E69002B90
:1085900008D12C4940398B6ACD042B438B628B6AFE
:1085A000AB438B62014631433CD025492368CB4223
:1085B00005D12449CA6803239B049A43CA6025460F
:1085C0002035002810D021680A6901231A430A6166
:1085D000216848610821204600F036F8032800D1C0
:1085E000A873216808204860002E10D02068016917
:1085F000012211430161206886611021204600F0AC
:1086000023F8032800D1A8732168102048600C4883
:108610002168C14206D10B48C168032292049143EC
:108620003943C16020680169490849000161216836
:108630000198886021680098C86062B6FEBD00009D
:108640000084FFBF4010024070B506460B480D463F
:10865000002409490068FCF74BFD7D21C90048430F
:108660003168401E00D103240B682A469A4301D08A
:108670000028F6D1204670BD204E00009C0100204D
:108680001CB5002116480091144A01910260C16393
:108690001205426081600722826301220261024664
:1086A000C16020321170FF235170C2334362816276
:1086B000117301638161042241634261C161FDF76D
:1086C00075FE084800908013019069460448FDF744
:1086D0001DFE00210248FDF7C3FD1CBD0024014022
:1086E000C01500200200000408B50848016B0122F3
:1086F00011430163006B01211040009000220A2009
:10870000FEF702FD0A20FEF7F3FC08BD0010024050
:10871000F0B587B014216846FCF749FD4748C26AA6
:1087200004210A43C262C26A0A400592C16A8026D5
:108730003143C162C16A31400591C16A01242143BC
:10874000C162C16A21400591C16A02252943C16203
:10875000C06A22462840059005201C210007FEF72C
:1087600044FA012236493748FEF73FFA00223649DB
:108770003448FEF73AFA9121052000220902000749
:10878000FEF733FA31480190002705206946029729
:1087900000940007FEF760F90C2000901120019072
:1087A000032003900520029769460007FEF754F95D
:1087B00010206A46039591C2052069460007FEF71E
:1087C0004BF91120019002976946039700941D48C8
:1087D000FEF742F91E480190694600950294194837
:1087E000FEF73AF9E00200906946019702951548B4
:1087F000FEF732F91748694691C169461148039757
:10880000FEF72AF991200002694691C105206946C8
:1088100000070397FEF720F969460A48019700967A
:108820000294FEF719F9002201210520FEF76CFCE5
:108830000520FEF75DFC07B0F0BD0000001002400F
:108840000102000000040050083000000000111078
:10885000000021100832000010B50F4C0D482060B8
:10886000FF20053060600020A060E0602061606152
:10887000E0610121206249026062A161A0620720DB
:10888000E0622046FFF78DF820680168402211431E
:10889000016010BD003001404C16002000B585B0CD
:1088A00014216846FCF783FC0E480D490160E12164
:1088B0004902416000218160C160016181610C2237
:1088C000C16142610162302141620121090381637A
:1088D0004900C163FFF77AFA01F04AFC05B000BD18
:1088E00000380140E416002070470000F0B589B060
:1088F0000A2002F08BFC7D20400102F0A1FCFF4C1D
:108900000025A570FE482066607C0C2801D30B2052
:10891000607460790A2801D90A206071F948E5700D
:10892000F94E00783071F949A07909784000084380
:10893000A17D89000843F071E06BF070010A31728B
:10894000401CE0636079B07442003046F049133057
:10895000FCF714FC6079EE49820040008019603118
:108960001330121DFCF70AFC6079062142004843CF
:108970008019E8491730921CFCF700FC2E20205E7D
:10898000002803D0E449098A0818E0856079DB49AA
:10899000C000223182190B7B53764B7B93760622E3
:1089A0007272DE4A1D301278B272A28C3273D64ACD
:1089B0000B79133A1375497951750022D24902F0A7
:1089C0000FFD60790021C0001D3002F01BFDD4486E
:1089D000FEF728FB01272085BF0309E0D048FEF7FA
:1089E00021FB80B22085E18EFF392D39884206DBDC
:1089F000E18E80B28842F1D3C9198842EED80220B4
:108A000002F054FCC0480126C571A574A5732674F4
:108A1000E573C348FEF706FB60850746E57060799D
:108A2000FCF74EFEBF4AC04BFCF72EFD01F038FEAE
:108A30000022BE4BFCF776FCFCF788FE0006C10C5A
:108A4000C81980B2F103A085884201D3401AA085DD
:108A5000B748E0642079401C2071B148FEF7E2FA83
:108A60002085AB48A54F643840370690B1E1AC484B
:108A7000FEF7D8FA20850BE0A948FEF7D3FA80B2BA
:108A80002085A18D884203D3AA4A8918884207D33A
:108A900000210F2002F03AFBA74920640842EBD0E6
:108AA000206C411C1FD040047ED58122D2010021C0
:108AB0000F2002F06AFC0021102002F027FB410683
:108AC0009348490E00227C38E16502F055FB0020F6
:108AD00002F0B6FB002002F068FB8D487C38417A3A
:108AE0000729C3D101E001F05FFC02229349401D38
:108AF000FCF768FB0028B9D102F0D5FCE167A0675C
:108B000002F0BEFC7D4B803303C3E0788049401CFB
:108B1000E07083390B7A68460370497A41700088A7
:108B20000390E18C88427DD1774985488C31C98E8C
:108B30000180754971488C31098F41847848FEF76E
:108B400071FA208502F0F4F96C48FF228030016848
:108B5000406852040023891858410206080A10434D
:108B60004108490000900A0E080264498031CA6039
:108B700088606548E36F0A30A26F02F069FC607993
:108B80008100614808185D49163080310CC902F037
:108B90005FFC5A488030C36882685B48123002F03C
:108BA00057FC0821584800E006E14172B430C07C0F
:108BB0000009607514D05648022260497738FCF7E6
:108BC00001FB00280CD15048A674C671E06D5049D5
:108BD0001638C2B26639C81DE274FB30FCF7CEFA13
:108BE00060790022800048491C3002F0F9FB60796E
:108BF000002180001C3002F005FC009802F0FFFA12
:108C0000012002F053FB207302214E48FDF7E0FFE4
:108C100000281DD000213D4801703B498C31488E11
:108C2000049000E05AE03881888E78818446A06CF8
:108C3000FF310531E0640860DC392065C97C090733
:108C4000090F032900D02175E16D1C2902D015E020
:108C50000121E0E72C49294A8C31C98F1186069BF6
:108C60002C4A1B881380884207DD002805DD002977
:108C700003D0207E401C207600E025762571A67367
:108C80000498B8816046F881E673608C2E49FF3005
:108C9000C33080B2608488420CD949424018608455
:108CA00027487D220188D200491C89B20180914267
:108CB00000D3058022487D210088C9004843618C8B
:108CC0004018606500F074FD207B002805D100216C
:108CD0000F2002F01BFA0006F9D583E0FDF72AF910
:108CE0000B4A03219032115407498C314A8E3A8144
:108CF000898E7981E26D1C2A2ED127E08800002020
:108D00003F420F005401002074120020880100200F
:108D1000A4130020E0140020400E00206401002075
:108D20001C160020B81E85EB51B8CE3F000008404D
:108D3000A0860100983A000000D027247801002086
:108D40008401002000040050E7030000614B420052
:108D5000D318069A12885A8080005F4B5E4AD43B33
:108D600002905D4982189B8F138030314118A26CAC
:108D70004A605A4940185A4916300CC902F068FB3B
:108D8000216EA06C884207DA534A02995158012992
:108D900002D12066039905914F49029A8958814270
:108DA00017DD012915DD2146002812DD0398C8844E
:108DB0000220087065730CE04A4A00210F2002F07F
:108DC000E4FA6079E178401C814202D0002002F090
:108DD000ECF9208DA18D884200D248E6424A8918DC
:108DE0008842FAD8A07B012801D00220A07302F0AB
:108DF0009FF83C4A00210F2002F0C7FA2079002892
:108E000017D03A4909888A008A18824200D2257010
:108E1000002000F0E5F8A07C002839D02E496C3104
:108E20000B78A372487860728A782272022B17D06E
:108E30002EE0E16C226E323920468A420EDAC17988
:108E40002A4A491CC9B2C171128852008A42E2D230
:108E50000599C184022101706573DCE7E571DAE7E9
:108E600010280CD0C82813D2214BC91C1818FCF7A5
:108E700085F903F027FA642001F076FC33E61D4DF6
:108E800028684000000E03D1C878FCF7FEFB28607C
:108E900000202378627B65790FE00F4E4100303E61
:108EA000775A1836765AB74205D00B4F0223002264
:108EB0000126483F7E52401CC0B2A842EDD3237029
:108EC0006273084A002180320F2002F05EFA09B076
:108ED000F0BD0000E0140020D41300207412002024
:108EE0000801002000D02724983A000064010020E7
:108EF000000E00207C010020F8B52E4C0546E06EE7
:108F00002D4A281A411E2067914215D21A21615E0E
:108F1000081AFCF7C1FB294A294BFCF7B5FA0646AB
:108F200032200F46205EFCF7B7FB32463B46FCF78B
:108F3000F9F9FCF7E7FB6086002060761D481C23EA
:108F4000C35E828C1F48008884461F4806881DE047
:108F50006046484380181D4F80B2388030277843E0
:108F60006427643078431A4F6066C01985420BD27B
:108F7000C8B2184932220880606EA25E411BC9182F
:108F80008918A166E066F8BD491C6176617EB14230
:108F9000DED33020424310486421101848430F4963
:108FA0004118E16660663221401B615EC0184018BE
:108FB000A066F8BD88000020CF0700009A99999913
:108FC0009999B93F720100206401002086010020B8
:108FD00078ECFFFF7001002074270000C0BDF0FF97
:108FE000FEB5294D2988491C8FB228492F800E884B
:108FF000FCF752FB264A274BFCF746FA01910090FA
:1090000025483146FCF774F8244C218F4218B742AA
:1090100006D3002028802248019E1018009D02E0FF
:109020001046019E009DFCF74BFB33462A46FCF799
:1090300079F9FCF78BFBA086012580B2ED03A842ED
:1090400001D3401BA086E08BFCF73AFB154A164B78
:10905000FCF782FA0646A08E0F460090FCF730FB24
:1090600032463B46FCF75EF9FCF770FB80B2E086C7
:10907000A84201D3401BE0860C490098096848616A
:1090800000982087FEBD00007001002064010020D0
:109090001904560E2D624040E17A0000880000203D
:1090A0001F050000F853E3A59B843E401C160020DA
:1090B00070470000F0B589B0002004900A2002F04B
:1090C000A5F87D20400102F0BBF8B3480022827071
:1090D000C16BB34C491CC163B049C38D098A254695
:1090E000C918C1852146C2751331079147310391D3
:1090F0006D393135AB4F223005910290A64E0F21CC
:10910000A948717100782071A84AB079127840009E
:109110001043B27D92001043E071B08FE070000AFE
:109120002072A17431461E229C310798FCF726F864
:10913000402228469E49FCF721F8029903980A7BB1
:10914000C274497B0175092060729A480078A07248
:10915000B08C2073F07D410030469C300918059892
:109160000A78027549784175762000228C4902F010
:1091700037F970790621484300211C3002F042F98A
:10918000022002F093F800210F2001F0BFFF3842C7
:109190003064F8D0306C411C18D040047ED5812258
:1091A000D20100210F2002F0F0F80021102001F080
:1091B000ADFF41067A48490E0022B43001F0DCFFD1
:1091C0007748B430417A022902D0BDE001F0ECF8D2
:1091D00002227949401DFBF7F5FF0028F5D16E48C2
:1091E0000222C07D41006C489C3009186C48B530A3
:1091F000FBF7E8FF0028E8D102F055F9664AD1678D
:10920000906702F03DF9644A803203C20498002856
:109210002CD1012004906248684E8C30C08E604989
:1092200030805D488C31098F41846548FDF7FAFE36
:109230005949644A0885488CFF30C33080B248845D
:1092400090420CD952428018488430885D4A401CB4
:1092500080B20B323080904201D3002030803088C1
:109260007D22D20050434A8C801848654C4869469C
:109270008C30428E0A80808E488049490422B53164
:10928000C81FFF38FBF77AFF4348494AC07D009961
:10929000800011504049803103C900E075E0FF2390
:1092A0005B040022C01851410906060A0E433046ED
:1092B00001F0A5FF710849000A0E08023649002690
:1092C0008031CA6088603448C36F826F3448483840
:1092D00002F0BEF8304880300CC83148443802F003
:1092E000B7F82D488030C36882682D48403802F0B6
:1092F000AFF82B49002252393C2002F071F80021CE
:109300003C2002F07FF8012001F0D0FF22490873D1
:1093100008468078401C887001210520C903000799
:10932000FCF71CFE1C48007B002805D100210F2003
:1093300001F0ECFE0006F9D5802200210F2002F09A
:1093400024F81548467002E013490120487012487D
:10935000C17D491CC9B2C1750F2900D2CEE604985F
:10936000002810D10C4A1849908C002802D00B8894
:10937000984201D908889084144980B20988401E17
:1093800048431349088009B0F0BD124A00210F205C
:1093900001F0FBFFD8E7000088000020400E00200D
:1093A0007412002000D027245401002088010020DE
:1093B0009014002064010020780100208401002026
:1093C0001C160020E7030000600100205E01002061
:1093D0005C01002000902724F8B53249304808602D
:1093E00002F014FA304800F0A3F9304CE0822E4825
:1093F000801C00F09DF920832B48001D00F098F997
:1094000060838B212A4889004180014640310979D7
:10941000284F0906090E617006D1C7800121C18756
:109420000A21418700218187234AC18E1170C18F93
:109430002171818F6171817AA170858805216562B2
:109440006181C6883046FBF753FEA081014628465D
:10945000FBF74EFE8800081885B216482581684340
:10946000FCF72EF9154A164BFCF776F8FCF76EF967
:10947000E081658231463846FBF73AFE208201469C
:10948000C820FBF735FEE0830120A083FCF76AFDCE
:10949000A082E2890B490C48FDF7C8FDF8BD000029
:1094A0009DA1000880000020004F0008540100200A
:1094B000000E0020E803000030000020F853E3A570
:1094C0009B843E40FF7F00001C160020F8B5754CC1
:1094D00000202071744D01202880744EC8203080F7
:1094E000E07A401CE072C00706D0A08C411EA18427
:1094F000022801D2C820A0840120C043FFF770FDDC
:109500000A2001F083FE7D20400101F099FE022136
:109510006748FDF75DFB00283FD0002065498000CB
:109520000978664F49000843634909780843B872CF
:10953000102078726248C1887D20C000FBF7D8FDFA
:10954000787360485E490078B87338460B308A7883
:109550000270C97841705A49421C20310B7ED37089
:10956000497E11715649D01C22310B7E5371497EC0
:109570009171534940310A7C0271497C417100224A
:109580003946172001F02CFF0021172001F03AFF87
:10959000022001F08BFE4C4F03E00120BEE7FEF7F6
:1095A00087FE00210F2001F0B1FD38422064F6D083
:1095B000206C411C73D040046FD58122D201002160
:1095C0000F2001F0E2FE0021102001F09FFD410676
:1095D0003A48490E0022B430E16501F0CDFD374F25
:1095E000B437787A112858D102223849781DFBF710
:1095F000E9FD002851D1F81F027A69460A70407AC5
:109600004870B97A2980C820FBF772FD3080387B1A
:10961000A08438462E4D2838C08E288039462148EF
:109620002839098F41842B48FDF7FCFC2085608C8C
:109630002949FF30C33080B2608488420CD9494246
:109640004018608428882449401C80B20B3128804F
:10965000884201D30020288028887D21C900484302
:10966000618C4018606500F0A3F868460088E084CB
:109670001249B87CC7316071420008460D46693016
:10968000FBF77CFD6079294642001448FBF776FD24
:10969000A08CFF2801D003202070F8BDFFE700F068
:1096A00083FE000088000020640100207201002079
:1096B00000040050580100205901002074120020BD
:1096C000000E00203000002000D027247801002068
:1096D000840100201C160020E7030000BC130020BA
:1096E00070B586B014216846FBF761FD01250F4E69
:1096F000ED03002229463046FDF777FA01200024C9
:10970000019002946946009503943046FDF7A4F950
:109710000320019002946946009503943046FDF7BA
:109720009BF9022001F020F806B070BD0004005043
:109730000088704770470000F8B5044600206A466C
:109740001080194D55222A70AA226A700322AA702D
:10975000661DEE702A716971144A49008918AC714E
:109760002246E81DFBF70AFD002007E029186A469B
:109770008978128889186A461180401CB042F5DB4E
:10978000611DA81CFCF74CFA0146684601802919A6
:109790000078C8716846407808722146093102484D
:1097A00000F012FBF8BD00005A150020000E00204A
:1097B000FEB5FFF7A1FB2548FDF734FC244C86B22B
:1097C000268560790A21081AC000FBF765FF074665
:1097D0000191A06EFBF774FF1E4A1F4BFBF7BCFE06
:1097E00000900D463046FBF76BFF2B46009AFBF7C7
:1097F00099FD3A46019BFBF795FDFBF7A7FF85B264
:10980000A586E08BFBF75CFF124A134BFBF7A4FE27
:1098100006460F462846FBF753FF32463B46FBF70A
:1098200081FDFBF793FF81B20120C003E1868142F5
:1098300001D3091AE186854201D3281AA08603497B
:10984000A08E096848612087FEBD00001C1600201C
:1098500088000020F853E3A59B843E40034A11682A
:10986000382389B2994301431160704700300140A9
:1098700010B5FDF7C7F910BD10B59AB03421684690
:10988000FBF795FC14210DA8FBF791FC1C2112A8F5
:10989000FBF78DFC1B4801680324E402A143C214BA
:1098A00089180160FDF73CFC17480169A14301617B
:1098B00006200090FF20013002900120039010202C
:1098C00004900220099040040B90000100240C90A9
:1098D0000A946846FDF752FE0F200D9003200E906B
:1098E0000F941094012111940DA8FDF71DFD812006
:1098F0001290032080041890149412A8FDF762FCC3
:109900001AB010BD007000404010024010480168BD
:10991000821511430160C1680E4A1140C16001689F
:109920000D4A114001608168490849008160016861
:109930000122920491430160C168FD221204914307
:10994000C160002101610649044888607047000039
:10995000001002400C40FF88F6FFF6FE00500008A1
:1099600000ED00E010B5CB06DB0E0121046A994042
:109970008C430462016A9A401143016210BD0000E9
:10998000F8B5102405252D07AC62AF20800000F04B
:10999000F2FEAC6101F0CEFB2F4C304F304E6067D1
:1099A0000EE001F0C7FB6067FEF782FC606C411CB3
:1099B0006164142804D92BA000F078FC2D48C760FE
:1099C000606FB042EDD10026666420780127FF0366
:1099D000030000F0A4FC05040C192D303200012214
:1099E00039462846FDF701F9FFF770FD06E0012230
:1099F00039462846FDF7F9F8FFF75CFB00223946A7
:109A00002846FDF7F2F818E0607B0122401C6073E5
:109A100039462846FDF7E9F8FCF7C0FA0022394636
:109A20002846FDF7E2F8607B052806D9267004E099
:109A3000FEF75CFF01E0FFF73DFB02210E48FDF75A
:109A4000C7F8002805D000200C49087001F058FA2A
:109A5000F8BD0120F8E70000880000200400FA05A6
:109A60003001CADE4457204944204552524F522EFD
:109A70000D0A000000ED00E0000400508801002005
:109A800010B5818CC90707D001684A6801235B04BF
:109A90009A43836A1A434A60818C890707D5016813
:109AA0004A6801231B049A43C36A1A434A60818CA3
:109AB000490707D501684A6801239B049A43036B51
:109AC0001A434A60818C090707D501684A68012357
:109AD000DB039A43436B1A434A60818CC90607D55E
:109AE0000268916801231B039943836B19439160BA
:109AF000818C890607D501688A6801235B039A4334
:109B0000C36B1A438A60818C490612D503685A6870
:109B100001210905046C8A4322435A60026C8A427F
:109B200007D10268516803235B059943436C1943CD
:109B30005160818C090607D501684A680123DB045E
:109B4000806C9A4302434A6010BD0000F8B5044699
:109B5000002680300660FDF74FF805462068006853
:109B6000124F000709D501212B4600224905204646
:109B7000009700F0A1FA00280DD120680068400786
:109B80000BD501212B46002289052046009700F0C5
:109B900093FA002801D00320F8BD2020A067E067D9
:109BA0002666603426750020F8BD0000FFFFFF0127
:109BB000F8B5154CC826E078002823D16079002834
:109BC00020D101206071114D686B0027002818D04A
:109BD000686BC821081A0FE00D48E168405C6169B4
:109BE0008847E068401CE060E068C82800DBE76068
:109BF000696BC820401A761EE168814201D0002EB0
:109C0000EADC6771F8BD00006C0000200000024033
:109C1000380D002070B5224CE07800283FD1207923
:109C200000283CD1012020711E4EF1690025090653
:109C3000002933DA2156625791420AD1F069400671
:109C40002CD5A079002829D0A5712089401C20811D
:109C500024E0A179002903D1A0710A2000F08BFD36
:109C600000202056CC2148430F4942182069121881
:109C70001279B262401C00222061A256CC235A43C2
:109C8000895881420ADC25612078401C20702078A8
:109C90000E2800D12570A078401CA070257170BDE1
:109CA0006C000020003801401002002010B5806ACE
:109CB0000022014640314A834A82FDF775FF10BDFC
:109CC00070B5846AA06FE56F21688968002609066F
:109CD000002906DA212804D152200653204600F03C
:109CE0006BF820688068400606D5222D04D15A20E2
:109CF0000653204600F047F82046803001681022C5
:109D0000114301602046FDF74FFF70BD10B50146BD
:109D10000968806A096889061CD400225A210A52FF
:109D200001680A68FF2301339A430A6001688A6860
:109D3000520852008A6001688A6840239A438A6008
:109D40002021C167016E012904D101680A6810232E
:109D50009A430A60016E012902D0FEF707F910BD8F
:109D60005821095AFDF71EFF10BD10B5806A016E1B
:109D7000012902D0FEF7FBF810BD5821095A490805
:109D8000FDF710FF10BD01680A68FF2321339A43D5
:109D90000A6001688A68520852008A60016E0129CF
:109DA00004D101680A6810239A430A602021C16720
:109DB000002101664166704701680A68C0239A4322
:109DC0000A6020218167704770B5164CE278002A3E
:109DD0000CD12279002A09D10122E2700025C8297C
:109DE00003DC0222A256002A01DCE57070BD0123CB
:109DF000E356CC2253430C4AD1500123E356CC26E0
:109E000073439B180A460146181DFBF7B7F96078A3
:109E1000401C607060780E2800D16570A078401EEC
:109E2000A070E2E76C00002010020020F8B50446A4
:109E3000016880682369E669184363690025334334
:109E40001843724A0B68724E334003430B6021681B
:109E5000486803231B039843E3681843486021685C
:109E6000A069914201D0236A18438B680B26360201
:109E7000B34303438B606749236867488B420CD127
:109E8000C0688007800F06D0012839D0022835D05D
:109E9000032821D11EE001271FE060498B420AD12F
:109EA000C0680C21084027D0042829D0082825D0D4
:109EB0000C2811D10EE093420ED1C168032080021C
:109EC000014019D001208002091A19D0091A15D0B1
:109ED000814201D1082700E010274F4950484039FE
:109EE0008600934232D1002F0CD0022F0DD0042FC8
:109EF00010D0082F7FD126E00027EEE70227ECE7FD
:109F00000427EAE7FDF7DEFA06E00968C90605D48A
:109F1000304603E0FDF7F6FA002872D0626851007F
:109F20005118814267D81103814264D3010E0602A1
:109F30005008002330185941FBF7F0F803210902BB
:109F4000411A384A55E00120C003E7E70122E369DE
:109F5000D20393422BD13B0000F0E1F90906090C32
:109F60004D114D4D4D274D00FDF7ACFA09E0FDF7C1
:109F7000B9FA06E00968C90605D4304603E0FDF7E2
:109F8000C1FA00283DD0616840004A088018FBF7FC
:109F9000AFF880B20146244A103991422BD8511CA7
:109FA00001400007400F084329E01046EBE73B0063
:109FB00000F0B5F90906090C211221212123210005
:109FC000FDF780FA0AE0FDF78DFA07E00968C90697
:109FD00006D4304604E00EE0FDF794FA002810D0D5
:109FE00061684A081018FBF783F880B201460E4AF0
:109FF0001039914203D9012503E01046F0E72168AA
:10A00000C86000206066A0662846F8BD0048004091
:10A01000F369FFEF00380140401002400044004067
:10A0200000093D00FFFC0F00EFFF0000F8B50446FB
:10A030004165403000262746028380373E6022205B
:10A04000E0672546206F603500281CD01749C162A3
:10A05000216F17480863216F16484863206F866395
:10A06000236F606D9C46134621680246604624318A
:10A07000FCF71AFC002806D0102038602E7520202E
:10A08000A0670120F8BD2E7520680168FF2201320B
:10A0900011430160206881680122114381602068BA
:10A0A00081684022114381600020F8BD0D9D0008A9
:10A0B0006B9D0008C19C0008FFB581B005460F46A6
:10A0C000044660350A9E39E0701C37D0FCF794FDD9
:10A0D0000499401AB04222D8002E20D0206801688E
:10A0E00049072BD5C069C043000527D4012021684A
:10A0F000C002086220680168FF22A132914301601A
:10A10000206881684908490081602020A067E067D5
:10A110008034206000202875032005B0F0BD206841
:10A120000168FF22A13291430160206881684908DB
:10A13000490081602020A067E067EBE72068C169E3
:10A140003846884305D0002103988142BCD00020C6
:10A15000E3E70121F8E7000010B504491020096881
:10A1600008620248FDF722FD10BD0000E416002041
:10A1700001490D20887070476C00002010B5FEF773
:10A18000B3FAFEF78BFBC82202490348FDF7BEFE77
:10A1900010BD0000380D0020E4160020F8B53E4C3C
:10A1A000002321783D4A1D46082910D0072947D0B1
:10A1B000062950D0052952D0042953D0032954D060
:10A1C000002956D0012958D002295AD05BE0A17845
:10A1D00000264A1F04E0314FBF5DFB189BB2761C7E
:10A1E0009642F8DB667927799A195118E3786278F4
:10A1F000C9188918C9194018C0430006000E1AD1A1
:10A20000012E14D0022E16D125482449C018FAF781
:10A21000B5FF02F057F8642000F0A6FABFF34F8FA5
:10A2200021492048C860BFF34F8F00BFFDE75908A0
:10A230001046FFF781FA2570E570A570A571F8BD8D
:10A24000A1795054491CC8B2A071A178491F884215
:10A25000F5D1082001E0607007202070F8BDE070A3
:10A260000620FAE760710520F7E7A070E57004208A
:10A27000F3E7552807D10120EFE7AA2803D10220F0
:10A28000EBE7032803D02570E570A570F8BD032027
:10A2900020702071F8BD00004C010020F614002051
:10A2A000000E00200400FA0500ED00E010B5024A9F
:10A2B000024900F0E5F910BD69B40008A0010020D2
:10A2C0002021020C01D010211046020A01D01046B4
:10A2D0000839020901D01046091F820801D0104632
:10A2E000891E420801D0881E7047081A7047F8B5C9
:10A2F000040C8BB2264682B25E430D0C1046370C1E
:10A300005843360480190021794116466E43370CB4
:10A3100036048019794126466E438919F8BD30B458
:10A320007446641E2578641CAB4200D21D46635DF2
:10A330005B00E31830BC18474900CA020243100012
:10A3400000D004204A0D01D001221043044A490DD7
:10A35000914201D102210843012800D10520704714
:10A36000FF0700008307FF22DB0E9A408907090ED2
:10A370009940002808DB830809489B001B181868CF
:10A3800090430843186070470007000F083883089F
:10A3900004489B001B18D86990430843D861704754
:10A3A00000E400E000ED00E0BFF34F8F04490348F4
:10A3B000C860BFF34F8F00BFFDE700000400FA053F
:10A3C00000ED00E0F8B504464F1EC800083821181B
:10A3D00015461E46086849683A4606239A4310D037
:10A3E0002A463346FBF750F83A46D200083AA318FB
:10A3F0001A687F1E5B68FAF795FF06223B46934377
:10A40000EED1022F23D0042F11D0062F2FD12A46B0
:10A410003346FBF739F8E36AA26AFAF783FF2A4664
:10A420003346FBF731F8636A226AFAF77BFF2A4664
:10A430003346FBF729F8E369A269FAF773FF2A4666
:10A440003346FBF721F863692269FAF76BFF2A4666
:10A450003346FBF719F8E368A268FAF763FF2A4668
:10A460003346FBF711F863682268FAF75BFFF8BD23
:10A47000002210B5134610460149FBF76DF810BDD8
:10A480000000F03F10B5FAF74DFF10BD002210B5E7
:10A49000134610461146FBF75FF810BD10B50721B3
:10A4A000024A00200907FBF7CFF810BD01030000A6
:10A4B000034A10B500201107FBF7C6F810BD0000D5
:10A4C00001FDFFFF02E008C8121F08C1002AFAD1EF
:10A4D00070477047002001E001C1121F002AFBD124
:10A4E000704700000149086070470000A401002087
:10A4F00008B50021684601706B46012202212C201C
:10A5000000F052FF0221684601706B4601222C20A8
:10A5100000F04AFF08BD000038B504466D206946CA
:10A5200008706B46012207492E2000F03DFF0649C6
:10A53000002C01D0054A00E0054A2E2000F01AFF49
:10A5400038BD0000060800000618000007060000DD
:10A550000716000038B504466B460222002136205B
:10A5600000F0EEFDB3212300FFF7D9FE0E0F081512
:10A570003A3A3A3A1C273A3A2F34483A0021684688
:10A58000017040784108490014E069460878800865
:10A590008000401C04E06946087880088000801C28
:10A5A00008701DE0684602780A404832027041781F
:10A5B000802001436846417012E0684602780A40F4
:10A5C000027040784106490EF4E769464878022156
:10A5D000084303E069464878FD2108406946487011
:10A5E0006B4601220021362000F0DEFE012200AB86
:10A5F00011463620013300F0D7FE38BD6946087891
:10A60000CF21084069462030CAE708B503216846D3
:10A610004170012101706B4602220021362000F0BA
:10A62000C3FE0122D20306212D2000F0A3FE01204B
:10A6300000F09AF80120FFF78DFF08BD08B5020A67
:10A6400069464A7008706B46022204212D2000F0F2
:10A65000ABFE0320694608706B46012206212D20BF
:10A6600000F0A2FE0020694608706B460122062118
:10A670002D2000F099FE0A212D2000F047FD08BD95
:10A68000F8B516460F460446002503E03946B047A4
:10A69000641C6D1C20780028F8D12846F8BD000005
:10A6A000F8B54A002B4B520DD6182B4A0C460546DE
:10A6B000142E2BDA002E12DA284BFAF733FE002282
:10A6C0001346FBF789F840D2002C03DA0124E40793
:10A6D00000253AE02046284337D0214C14E0214F92
:10A6E0000B46F7403B402B4331D01C4BFAF71AFE88
:10A6F00000221346FBF770F827D2002C03DD01205F
:10A700000005F0400419BC4300251EE0332E1EDC7A
:10A7100033460027143BFF43DF40384217D00F4B2E
:10A72000FAF7AAFE00221346FBF756F80DD2002CCA
:10A730000ADD142E0CD03420811B012088404019E2
:10A74000A84200D2641C0546BD4321462846F8BDF8
:10A75000641CF9E701FCFFFF9C7500883CE4377E30
:10A760000000F03FFFFF0F007D2110B5C9004843F6
:10A7700000F001F810BD002140E000BF00BF00BFA5
:10A7800000BF00BF00BF00BF00BF00BF00BF00BFD1
:10A7900000BF00BF00BF00BF00BF00BF00BF00BFC1
:10A7A00000BF00BF00BF00BF00BF00BF00BF00BFB1
:10A7B00000BF00BF00BF00BF00BF00BF00BF00BFA1
:10A7C00000BF00BF00BF00BF00BF00BF00BF00BF91
:10A7D00000BF00BF00BF00BF00BF00BF00BF00BF81
:10A7E00000BF00BF00BF00BF00BF00BF00BF00BF71
:10A7F00000BF00BF00BF00BF00BF491C8142BCD3E7
:10A800007047FFB581B01E460F46040026D00B9955
:10A8100003980143A06A39438268072090470028C3
:10A8200018DB0A99A06A3143826806209047002805
:10A8300010DB25462035A979032F01D908200143D3
:10A84000032E01D904200143A06A826809209047A1
:10A85000002806DA0120C04305B0F0BD0020C04347
:10A86000FAE7384600F000F92060304600F0FCF8C6
:10A8700060600A9868700398A870EF702E710B984A
:10A8800068710020E8E70000F7B50446002090B0AA
:10A8900000900190002C05D06A46062101F04CFD85
:10A8A000062803DA0020C04313B0F0BD68464078A4
:10A8B0000102684600780004091868468078081884
:10A8C000FAF7FEFE054668460391007901026846E4
:10A8D000C07800040918684640790818FAF7F0FEB5
:10A8E000032206460F4692075C4BFAF775FF07D224
:10A8F00000225B4B30463946FAF7B8FD06460F4654
:10A9000003229207554B28460399FAF765FF07D2B1
:10A910000022534B28460399FAF7A8FD05460391F8
:10A920002068FAF7CDFE02460B4630463946FAF764
:10A9300013FE07460A200791205EFAF7ADFE3A465D
:10A94000079BFAF7A1FD064608200991205EFAF759
:10A9500091FE0021C943FAF7D9FCFAF715FF3246F8
:10A96000099BFAF7DFFC069108906068FAF7A8FEE9
:10A9700002460B4628460399FAF7EEFD05461A20D3
:10A980000E46205EFAF788FE2A463346FAF77CFD2B
:10A990000C9009911620205EFAF77EFE099B0C9A16
:10A9A000FAF7C0FC05910A902A46334638460799C3
:10A9B000FAF76AFD059B0A9AFAF766FD05910A9077
:10A9C0001420205EFAF768FE3A46079BFAF75CFD12
:10A9D00007461C200791205EFAF75EFE2A463346A2
:10A9E000FAF752FD0E900B911820205EFAF754FEF4
:10A9F0000B9B0E9AFAF796FC2A463346FAF744FD6B
:10AA00000B910E902069FAF747FE0B9B0E9AFAF70E
:10AA100089FC2A463346FAF737FD05460E46E068BC
:10AA2000FAF73AFE2A463346FAF77CFC3A46079B89
:10AA3000FAF778FC059B0A9AFAF774FC0122920750
:10AA4000084BFAF721FD02460B46129C089806991E
:10AA500003C411980CC0002026E70000FFFF5F41EF
:10AA600000007041E17A843F00B50121C904030070
:10AA7000FFF755FC081A05080B0E1114171A0320CE
:10AA8000C00400BD0720C00400BD0F20C00400BDED
:10AA90001F20400300BD3F20400300BD7F20400336
:10AAA00000BDFF20400300BD084600BDFEB5264F97
:10AAB0000D4604000FD0002D0DD026460020203674
:10AAC000B071F07129680D208847002801DA7800FC
:10AAD000FEBD102801D03846FEBDA562E9680029F8
:10AAE00001D028208847204600F030F80028F3DB0A
:10AAF000A06AA52182680E209047A06A96218268EC
:10AB00000F209047A06A0221826862209047A06AC5
:10AB1000002182680E209047A06A002182680F20E1
:10AB20009047717930200191009006232022012165
:10AB30002046FFF766FE0028CEDB204600F0AEF888
:10AB40000028C9DB0020FEBDFFFFFFFF10B586B067
:10AB5000044614216846FAF72AFB002C7ED0A06A2E
:10AB6000122143686A4610209847122877D1684618
:10AB70000078012201016846407812030009081894
:10AB800043492081884201DD801A2081684683780C
:10AB900040780007000D18186081884201DD801A96
:10ABA000608168460079012201016846C07812057B
:10ABB0000003091868464079000908183549E06023
:10ABC000884201DD801AE060684640790007030B87
:10ABD0006846807900021B186846C0791818206101
:10ABE000884201DD801A20616846417A007A0002BD
:10ABF000081802B2284801210904A282824201DD1C
:10AC0000521AA2826A46D37A927A12029A1812B221
:10AC1000E282824201DD521AE2826A46537B127B53
:10AC200012029A1812B22283824201DD521A228342
:10AC30006A46D37B927B12029A1812B262838242D6
:10AC400001DD521A62836A46537C127C12029A1802
:10AC500012B2A283824204DD501A01E00BE008E048
:10AC6000A083A06A016828208847002806DA01200E
:10AC7000C04306B010BD0020C043FAE7C011C007B2
:10AC80002034002800D0802060710020F1E700000F
:10AC9000FF070000FFFF0700FF7F000010B5040062
:10ACA00009D0A06A0721826808209047002805DAA9
:10ACB0000120C04310BD0020C04310BD0720203438
:10ACC0002070002010BD0000FEB504460020019059
:10ACD00000906079734940000E5A61782578491ECA
:10ACE0007148CFB20163042D77D0072D75D00021B4
:10ACF0000291217801736C49E379012292058969F7
:10AD0000002B6CD0914381616748217A4173217A8D
:10AD100082698907890B0A4382610021042000F0BF
:10AD200034FB324661492E2000F024FB3846FFF701
:10AD3000F3FB5F4E0522705D810040185D494318AA
:10AD400007212B2000F030FB5B49029801220B18F1
:10AD50000B21282000F028FB705D584980000A581C
:10AD60000C21282000F011FBE079554980004018A3
:10AD7000A1794900425A0221272000F0FBFA5148EC
:10AD80007E00825B0421272000F0F4FAE07900289D
:10AD900029D0A07804282CD02820694608722022C7
:10ADA0000621272000F0E6FA02AB01222621272007
:10ADB00000F0FAFA444938014018E1788900425815
:10ADC0000821272000F0E1FAA17A601C627A0902CA
:10ADD000114313D016E000E001E0012188E71143A0
:10ADE000F608816190E764220621272000F0C2FA6C
:10ADF000E0E71020694608720246D1E73349017244
:10AE0000090A4172417A007A0A020243202127206E
:10AE100000F0B0FA2E4F0C2123203A6800F0B5FA6A
:10AE2000F01982880421232000F0A4FAA0790028D8
:10AE30000BD0E0792749012243180021212000F09E
:10AE4000B3FA03200190012000902A07120F10018D
:10AE50000243607800218007000B0243019800053F
:10AE600002430098400402432079C006400902438F
:10AE70006079C00602431F2000F087FAA07861784D
:10AE80000123084302040848DB030261E179490316
:10AE900019430A4302610021082000F076FA0020DD
:10AEA000FEBD00006CC40008D4010020042800008E
:10AEB00014C400083C0000205A0000201CC40008F4
:10AEC0003CC4000848C400084CC4000841100000FD
:10AED00034C400085C00002038B50C4607498A8B52
:10AEE000002102432C2000F045FA684604706B46AE
:10AEF000012206212C2000F057FA38BDD401002091
:10AF000010B5FFF7F5FA10BD10B504460421362040
:10AF100000F0FCF80121C902002C01D0084300E038
:10AF2000884302460421362000F02FFA10BD0000AD
:10AF300038B540206946087000210E2000F0E6F880
:10AF40000446002211460E2000F01FFA6B46012233
:10AF500000210D2000F028FA074A00210F2000F000
:10AF600014FA00F0EDF9224600210E2000F00DFA4F
:10AF700002480021017338BDF8FF2724F4010020A6
:10AF8000FEB50546042069460870514C00206075E6
:10AF900021462031206348710873A0836063A06359
:10AFA00000F0C8F84B4E206002E000F0C3F82060CB
:10AFB000B042FAD10020FFF7CDFA00F0BBF8464EC0
:10AFC00020603078242801D9243806E00621FAF7D9
:10AFD0008FF80622101A40010843020601040A43B2
:10AFE00001020A430243B260706000211E2000F09B
:10AFF000CCF900F09FF820606B460122002124204C
:10B0000000F0D2F91E20FFF719FB86B2300AA073B8
:10B010000420FFF713FB074600F08CF82060380689
:10B02000000E0DD002206946087101AB01221221E9
:10B030002D2000F0B9F9A08B012109030843A0835A
:10B0400000F078F820600620FFF7F8FA606007202B
:10B05000FFF7F4FAA060F006C00E207501D11020B1
:10B060002075C0B200F0DCF9E80707D0FFF7CDFA91
:10B07000A08B0121C9020843A0830AE005213620E4
:10B0800000F02EF81549084002460521362000F050
:10B0900071F90120FFF75EFA0021042000F036F874
:10B0A000A0610021262000F031F815218903084312
:10B0B00002460021262000F068F9002226213620D1
:10B0C00000F058F900F036F820600020FEBD0000C6
:10B0D000D40100203001CADE30000020FFFD000056
:10B0E00038B5094C89B280B26B46022200F028F8CC
:10B0F000002806D1684640780102684600780818A2
:10B1000084B2204638BD0000FFFF000038B500249F
:10B11000E44389B280B26B46042200F011F80028A3
:10B1200006D103216846435C2202D418491EFAD591
:10B13000204638BD10B500210846FFF7E7FF10BDD7
:10B1400038B5002909D0402420436C462070C8B28D
:10B150007F2906D8607002200AE069460870012045
:10B1600006E0802420436C466070C809A07003206C
:10B17000694601F081F838BD10B5144603460A4609
:10B1800021461120FFF7DCFF10BD10B50346052254
:10B1900000211520FFF7D4FF10BD10B5034605228E
:10B1A00000211720FFF7CCFF10BD38B50546002061
:10B1B0006946087000F0C4F8FF2401342246002DCF
:10B1C00001D00322120200210D2000F0D3F8002D3F
:10B1D00013D06B46012203210F20FFF7B1FF684611
:10B1E0000078000709D5FFF7A3FE224600210D20B5
:10B1F00000F0C0F80020C04338BD002038BD10B5B5
:10B20000024601210A2000F0C0F810BD10B5044626
:10B2100000211A20FFF77AFF000D22030005120B10
:10B22000024300211A2000F0B0F810BD10B502460C
:10B2300002492E2000F09EF810BD00000418000006
:10B24000F8B505466B46012203210420FFF778FF7D
:10B250000126114C3607002D0DD02A4600210C2066
:10B2600000F088F86946087810210843694608709C
:10B27000A069304307E069460878EF210840694635
:10B280000870A069B0430B46A0610122032104208D
:10B2900000F08AF8F8BD0000D401002010B5024685
:10B2A0000021182000F066F810BD0000F8B5074630
:10B2B000002568460570B807204C2E4600280ADA9B
:10B2C0008020694608706B46012200210D2000F0A5
:10B2D0006BF801202073F8076946087821D0062111
:10B2E0000843694608706B46012200210D2000F0DA
:10B2F0005BF803210F20FFF7F3FE8121C90008420C
:10B3000019D04020694608706B46012200210D20AB
:10B3100000F04AF80020FFF7F7FD00252673ED4303
:10B3200009E002210843694608706B4601220021AA
:10B330000D2000F039F82846F8BD0000F401002087
:10B340001CB56B46012203210F20FFF7F9FE68466A
:10B3500000784022C1091040C9014000814208D054
:10B36000012069460871024601AB03210D2000F05F
:10B370001BF81CBD08B56B461A70120A5A7089B2C8
:10B3800080B2022200F010F808BD38B500236C46E8
:10B39000E254120A5B1C042BFADB89B280B223460A
:10B3A000042200F001F838BD38B58024002909D006
:10B3B000C02528436D462870C8B27F2907D8687019
:10B3C000022009E0204369460870012004E0204380
:10B3D0006870C809A8700320694600F0F7FF38BDFF
:10B3E00010B51446012312189B029A4202D900207C
:10B3F000C04310BD0B46821E21460920FFF7D4FF33
:10B40000002010BD10B5054A8905126901430A43A1
:10B4100000210820FFF7B9FF002010BDD401002053
:10B4200038B504466B4601220E212B20FFF788FE1B
:10B4300068460078E10640094001C90E01436846AC
:10B4400001706B4601220E212B20FFF7ADFF38BDA6
:10B4500010B5002142541C06120A22431B0A491C43
:10B460000429F7DB10BD000013B501231A46694615
:10B470000248FCF77DFD00981CBD0000E41600208A
:10B480007CB5002425466846FFF77FFE0420694608
:10B49000220E2D02154322020C5C1443401EF7D5E8
:10B4A000204629467CBD7CB5002425466846FFF72A
:10B4B00074FE04206946220E2D02154322020C5C04
:10B4C0001443401EF7D5204629467CBDFBF7A2FB5E
:10B4D000FEF7D2F9FDF71CF93E493F48002522C08E
:10B4E00005608561C5613D490562C1600838FBF7AB
:10B4F00023FDFDF7F9F8FDF7D1F9FDF7ADF9FDF7FB
:10B50000BFF8052401222407D1032046FBF76DFB79
:10B51000FDF762FFFAF742FBFAF75EFBFAF7E0FB92
:10B52000FAF7AEFBFCF7A6FD0721A015FFF7D4FC48
:10B53000FFF7E6FC012211032046FBF756FB2648E5
:10B54000C8222749C830FCF7E1FC264F264E274C7D
:10B55000387800280FD13078002801D003280AD18C
:10B560000121C9022248FBF733FB002803D1012146
:10B570000846FBF7F5FDE078002828D06078002821
:10B5800025D0E57072B620780F280AD90120184915
:10B5900000038861FEF7F4F9012015490003886271
:10B5A0000CE0012251031248FBF71FFBFEF7E8F9FC
:10B5B0000121002249030E48FBF717FB62B6FCF796
:10B5C00077FE208C0028C3D0401E2084C0E7FCF703
:10B5D0006FFEBDE7007C00401C160020FFFF00004E
:10B5E000380D0020720000209C0000205401002033
:10B5F0000004005010B586B01748FBF720FC14215A
:10B600006846F9F7D4FD154800900320019000200A
:10B610000290052069460007FBF71EFA69461048AC
:10B62000FBF71AFA69460F48FBF716FA012108469C
:10B63000FBF796FDFF2401342046FBF769FD0A491C
:10B6400008680422104308602046FBF771FDFBF7F1
:10B6500077FD06B010BD00001C160020FFFF0000A3
:10B6600000040050000800500070004010B504466F
:10B67000FCF7BAFD4E20FCF78AFDFCF7EEFDE0B2C8
:10B68000FCF785FDFCF7E9FDFCF7AEFD4F20FCF76C
:10B690007EFDFCF7E2FD0020FCF74CFD0446FCF7C4
:10B6A000BEFD204610BD70B50D460446FCF79CFD5E
:10B6B0004E20FCF76CFDFCF7D0FDE0B2FCF767FD17
:10B6C000FCF7CBFD2846FCF762FDFCF7C6FDFCF756
:10B6D000A6FD0A20FFF74FF870BD000010B5242129
:10B6E000002000F04DF81B48FFF745F800210F201F
:10B6F00000F046F80521102000F042F80421112046
:10B7000000F03EF883217F2000F03AF869217F2085
:10B7100000F036F8BD217F2000F032F80E480078A6
:10B72000262804D1002240218C2000F019F80120A5
:10B7300000F02AF8094814210187282000F020F899
:10B740000A20FFF718F8012000F036F8012000F079
:10B7500043F810BD204E000000000020000E002025
:10B76000F8B517460E4605460024FFF77FFF394619
:10B77000B44331402143284600F002F80020F8BDD0
:10B7800010B5FFF790FF10BD10B500280AD00021BA
:10B790002720FFF7F5FF04211920FFF7F1FF87218C
:10B7A000162005E000211620FFF7EAFF00211920EE
:10B7B000FFF7E6FF10BD000010B5002801D0002201
:10B7C00000E0802280211120FFF7CAFF0148FEF728
:10B7D000D2FF10BDA086010010B5002811D00121B4
:10B7E0002F20FFF7CDFF62213020FFF7C9FF462150
:10B7F0003120FFF7C5FF32210846FFF7C1FFA22124
:10B8000000E022213320FFF7BBFF10BD10B501225D
:10B81000920217491748FAF7E7FA154816490288BD
:10B820008A4223D0018004218180FF21F531C1802B
:10B830000A21018100211E224181D24382810122FD
:10B84000C28181834323C3860223038778234387EE
:10B850008287C28702464032118451849184C18319
:10B86000918014238382118200F02CFD10BD000012
:10B87000000E002000FC0008AA550000F0B51FB41F
:10B8800096B084460C460246199D189803904900CC
:10B8900068006300490840080193002A01D001268E
:10B8A00000E000269E19FE4BF6185B109E422BD33B
:10B8B0006E00039F0296002F00D00127F719F84E63
:10B8C000F84BBE199E421FD3039E0346F64F3343E7
:10B8D00009D03B469C4201D1002A04D0019B002A9A
:10B8E00005D0012604E0002039461BB0F0BD00263B
:10B8F0009E19EE4B9E4207D8039F029E002F00D058
:10B900000127F6199E4207D92B4660462146189A10
:10B91000FEF7B8FD1BB0F0BD0023002C29DAE44E81
:10B92000B04226DAE34EB04201DB022321E0DE4ED4
:10B93000B0421EDBE04E070DBE19142E09DD342780
:10B94000BF1B039EFE400196BE40039FBE420BD02C
:10B950000FE0039F002F0CD11427BF1B0646FE40AB
:10B960000196BE40864204D1019BDE07F60F0223FA
:10B970009B1B0E46164318D1002D16DA002C03D05F
:10B98000022B01D0012B06D00220FEF7ABFDFEF703
:10B990006FFD1BB0F0BD0220FEF7A4FDFEF768FDB1
:10B9A0000122D20751401BB0F0BD039E002E61D191
:10B9B000BF4EB04220D1C148844201D1002A08D0F4
:10B9C000B948814209DB002D10DB189829461BB0CD
:10B9D000F0BD0020B4491BB0F0BD002D06DA0122F5
:10B9E0002946D207189851401BB0F0BDB44979449C
:10B9F000086849681BB0F0BDAB4FB84225D1002D97
:10BA00001FDA002904D0B14212D1002A09D018E06F
:10BA1000002A72D1A649E20F0020D20711431BB0C1
:10BA2000F0BD0020E20F0146D20711431BB0F0BD6C
:10BA3000B14206DA234600203946F9F78DFD1BB0E6
:10BA4000F0BD104621461BB0F0BDB14212DA01260E
:10BA5000B607B54203D1234610461946FEE3994E78
:10BA6000B54207D1261E05DB1046314600F040FCEA
:10BA70001BB0F0BD67007F081646002A40D10029A0
:10BA80000AD08B4A914229D1002C0EDD002D1CDBFF
:10BA9000002011461BB0F0BD022B16D0002C14D094
:10BAA000012B12D1002C14DB0FE0002C28DA002D22
:10BAB00009DB012B03D000207D491BB0F0BD002025
:10BAC00081491BB0F0BD012B03D0002001461BB003
:10BAD000F0BD00200121C9071BB0F0BD724A9142A0
:10BAE0000ED1002C01DA002B17D0022B06D000203B
:10BAF000C043F9F7D1FD1BB0F0BD90E20120F8E79B
:10BB0000E217521C94461A4307D000220892664C52
:10BB100062465B1E1A4307D009E00120FEF7E2FCF3
:10BB2000FEF7B4FC1BB0F0BD0022644C0892674ADB
:10BB300090427DDD664B674A98421FDD914202DCF0
:10BB4000002D05DB4DE05848814217DB002D48DD14
:10BB50000220FEF7C7FCFEF7A1FC05460E460022B8
:10BB6000534B21460898F9F78FFC084671004908A5
:10BB7000C00FC007014328461BB0F0BD914215DA43
:10BB8000002D2EDA0220FEF7ADFCFEF787FC0546FD
:10BB90000E460022464B21460898F9F775FC7200C4
:10BBA0005208C80FC0070243114617E03E4B9942A6
:10BBB00023DD002D15DD0220FEF794FCFEF76EFC60
:10BBC00005460E4600223A4B21460898F9F75CFCE0
:10BBD000084671004908C00FC007014328461BB042
:10BBE000F0BD0220FEF77EFCFEF762FC490049082A
:10BBF000E20FD20711431BB0F0BD00223046394698
:10BC0000F9F734FC012205460E46D243F9F71CFD34
:10BC1000314A324BF9F730FC2A463346F9F734FC07
:10BC20000022284BF9F728FC07462A46334600E055
:10BC300064E0039110461946F9F726FC3A46039B47
:10BC4000F9F722FC0746032209915207244B2846A4
:10BC50003146F9F719FC07910C90224A204B3846DF
:10BC60000999F9F711FC074601911F4A1F4B284615
:10BC70003146F9F709FC3A46019BF9F7F7FB07460D
:10BC80000B460246099107990C98F9F74BFB0025E2
:10BC90000E462846079B0C9AF9F7E8FB3A4627E040
:10BCA000FFFF1F00FFFF0F000000F03F0000E0FF5C
:10BCB0000000F07F0000404301FCFFFF0000F0BFE8
:10BCC000560B00000000E03F0000F0FF0000E041E4
:10BCD0000000F043FFFFEF3F555555555555D53FF3
:10BCE0004715F73FFE822B6544DF5DF80BAE543EEF
:10BCF000099BF9F7C1FB02460B4652E101250020E2
:10BD00002D05A94207DA352230463946F9F79CFC61
:10BD100006463420C0430A151218FE481018039036
:10BD20000803FD49000B01430F46FC49884201DC32
:10BD3000002003E0FA49884202DA0120119005E070
:10BD4000002011900398401C7F1B039011980597C9
:10BD5000C200F4480F92784480184368026839465C
:10BD600030460D930292F9F781FB07910C90304613
:10BD70000D9B029A0599F9F7D5FA02460B46002069
:10BD8000E549F9F7E9FB09910490079B0C9AF9F74B
:10BD90007BFB129000201090E3480D467844006829
:10BDA0000E90012178104907084311990D9B8904D1
:10BDB00040180121C90447183946029A0E98F9F72C
:10BDC00055FB3246059BF9F757FB02460B462946C1
:10BDD0001098F9F759FB064602913B4629460E9A00
:10BDE0001098F9F751FB079B0C9AF9F745FB32467F
:10BDF000029BF9F73BFB099B049AF9F745FB059178
:10BE0000129A0A902B4610461946F9F73DFB064652
:10BE10000246C6480F460B4606217844FEF7D2FA82
:10BE200032463B460091049010461946F9F72CFB28
:10BE3000009B049AF9F728FB06460F462B46194645
:10BE4000129A1098F9F76EFA059B0A9AF9F71CFBFB
:10BE500032463B46F9F766FA109A079104902B4652
:10BE600010461946F9F710FBB14E002233460991EE
:10BE70000290F9F757FA079B049AF9F753FA002052
:10BE80000746024633460091F9F7F0FA099B029AF9
:10BE9000F9F7ECFA079B049AF9F7EEFA06460D91CA
:10BEA0003A462946009B1098F9F7EEFA07910C9054
:10BEB0002B463046129A0D99F9F7E6FA05460E46DA
:10BEC0003A46009B05990A98F9F7DEFA33462A4666
:10BED000F9F728FA02460B460746099107990C988C
:10BEE000F9F720FA00250E462846079B0C9AF9F729
:10BEF000BDFA3A46099BF9F7BFFA074607220991AE
:10BF000052078C4B31462846F9F7BEFA079100904C
:10BF1000894A884B38460999F9F7B6FA07460191DC
:10BF2000864A874B31462846F9F7AEFA3A46019BD6
:10BF3000F9F7F8F9834B7B440F9A9B181A685B68F2
:10BF4000F9F7F0F9029009910398F9F7A5FB05912B
:10BF50000490099B029A07990098F9F7E3F97A4B44
:10BF60007B440F9A9B181A685B6817460393F9F78E
:10BF7000D9F9059B049AF9F7D5F90E462846059B91
:10BF8000049AF9F773FA3A46039BF9F76FFA079B9D
:10BF9000009AF9F76BFA099B029AF9F76DFA0246D3
:10BFA0000B46199900200C900F461898F9F76CFA77
:10BFB000029104903B460C9A19991898F9F756FA91
:10BFC0002A463346F9F760FA029B049AF9F7AAF970
:10BFD00009910E902A46334639460C98F9F754FADF
:10BFE00006460F46099B0E9AF9F79CF9574A0D46EB
:10BFF000914220DB5242AA18024310D132463B46FE
:10C00000F9F734FA04900391514A524B09990E986A
:10C01000F9F788F9039B049AF9F7DEFB1ED2022098
:10C02000FEF760FAFEF73AFA49004908E20FD20734
:10C0300011431BB0F0BD6A00474B52089A420DD322
:10C04000464AAA18024300D0CBE532463B46F9F7F0
:10C050000DFA099B0E9AF9F7BFFBF5D9680000238A
:10C0600040082C490393020D3D4B5218984223DDA2
:10C0700001200005521CD04042195000400D4018CC
:10C0800038497944096813468C463749C1408B4387
:10C0900012030121120B090551181422101AC14074
:10C0A0000391002D01DA484203906246304639463A
:10C0B000F9F7DCF906460F4632463B4609990E98D9
:10C0C000F9F730F900252A46284B28460591F9F75B
:10C0D000DBF907910C90264A264B28460599F9F77B
:10C0E000D3F90091029032463B4628460599F9F76C
:10C0F000BDF9099B0E9AF9F7BFF91F4A1F4BF9F7D3
:10C10000C3F9009B029AF9F70DF907460B46024660
:10C11000099135E001FCFFFF0000F03F8E9803001D
:10C120007AB60B0066070000A8070000D2060000E0
:10C130000000084009C7EE3FFD033ADCF5015B143F
:10C14000E02F3EBEA60500006C05000000009040F8
:10C15000FE822B654715973C00CC904000346F3F22
:10C160000000E03FC2040000FFFF0F00432EE63F47
:10C17000396CA80C615C20BEEF39FAFE422EE63F16
:10C1800007990C98F9F7CEF805460E46079B0C9ACE
:10C19000F9F76CF93A46099BF9F76EF909912A46C5
:10C1A00033460E9010461946F9F76EF907460246D7
:10C1B0002F480B46059105217844FEF703F93A46CE
:10C1C000059BF9F761F92A463346F9F755F9074611
:10C1D000019128463146099B0E9AF9F755F9099BBA
:10C1E0000E9AF9F79FF8012304910C9000229B0707
:10C1F00038460199F9F73AF905910E903A462846E2
:10C200003146019BF9F740F9059B0E9AF9F7A4F91D
:10C21000049B0C9AF9F72AF92A463346F9F726F9CE
:10C220000022144BF9F728F9064603980D4600053D
:10C2300041190915002912DC30462946039AF9F7FD
:10C2400003FAFEF779F8042801D1FEF731F93046F8
:10C250002946039AF9F7F8F9064601E004E029189F
:10C260000B46324621460898F9F70EF91BB0F0BD8F
:10C27000640300000000F03FF0B58C460025102656
:10C28000052109078E620E4C08E067467F5DE76076
:10C29000A768FF07FCD0E7681F706D1C8542F4DBC0
:10C2A0000020074606E0E760A568ED07FCD0E568DA
:10C2B0001D54401C9042F6D38E610020F0BD00005A
:10C2C0000030014070B572B60124074DA40221462A
:10C2D0002846F9F76FFD002804D022460349284676
:10C2E000F9F70CFE62B670BD00FC0008000E0020DD
:10C2F000F8B506460C46F9F77DFB051E0F4600D043
:10C300000120014349000B484908411AC90F0DD0CB
:10C31000002E01D0012100E000210C4361004908FA
:10C32000401AC00F02D10120FEF7DCF8284639463A
:10C33000F8BD00000000F07FF8B515460E46074630
:10C34000002407E03819C0B200F008F8641C287017
:10C35000E4B26D1CB442F5D33046F8BD10B50446C6
:10C36000FBF742FFEE20FBF712FFFBF776FF2046BC
:10C37000FBF70DFFFBF771FFFBF736FFEF20FBF735
:10C3800006FFFBF76AFF0020FBF7D4FE0446FBF72D
:10C3900046FF204610BD704770B50D460446FBF7BA
:10C3A00023FFEE20FBF7F3FEFBF757FF2046FBF7DA
:10C3B000EEFEFBF752FF2846FBF7E9FEFBF74DFFC9
:10C3C000FBF72DFF0A20FEF7D6F970BDF0B500256A
:10C3D000102605279C463F070B46BE620C4C06E024
:10C3E000595DE160A168C907FCD0E1686D1C854218
:10C3F000F6DB002007E06146095CE160A168C9073F
:10C40000FCD0E168401C9042F5D3BE610020F0BD35
:10C41000003001400000010203040005405C000000
:10C42000A05C0400C06C0800805C0400E03F1E00BB
:10C43000E07D1E0007A9022570889B880A0016006F
:10C44000010006000100020087008D002D001A3156
:10C4500052001A339A001A351D011A376B003B310E
:10C46000BE003B335E013B3596023B3700009959D5
:10C470009959EB518F421E45142E0080EB51F5283F
:10C480003333E13A703DE13AC235852BC23533335F
:10C49000C235C235AE47E13A5138A33051380000B9
:10C4A000000000000000010203040607080903045D
:10C4B00006080C10182030000000000102030400E0
:10C4C000000000000000F03F000000000000F83F06
:10C4D00000000000000000000000004003B8E23F40
:10C4E000000000000000000006D0CF43EBFD4C3EF2
:10C4F000033333333333E33FFFAB6FDBB66DDB3FE7
:10C500004D268F515555D53F01411DA96074D13F2E
:10C5100065DBC9934A86CD3FEF4E454A287ECA3F28
:10C520003E5555555555C53F93BDBE166CC166BFAA
:10C530002CDE25AF6A56113FF16BD2C541BDBBBEA3
:10C54000D0A4BE726937663E000000000000000003
:10C5500070C5000800000020A8010000BC5A0008B7
:10C56000D4C50008A8010020681A0000D4A400085F
:10C57000023B27130704380D091E08054008260949
:10C58000104008560A131D043B08BE0516D8BC40CF
:10C5900010085201033AC842077052030CE5800CA0
:10C5A0001B0202DD140901022281F01F668104983A
:10C5B0008996869679821598039814988796749729
:10C5C0007882439788967197778249F10139293F9C
:04C5D000920492201F
:04000005080050C1DE
:00000001FF
